:020000041100E9
:10300000002373B52B4D2C4C28006361022601F080
:103010006BF94021FE2221742800284B009601F014
:10302000B5F9002836D1217CFF222800244B0096D8
:1030300001F0ACF900282DD1224BA2899A4226D169
:10304000E389214A93420DD1204B6361204B2268D2
:10305000002A03D1002B01D043CB43C4280001F048
:1030600081F973BD1B4A934201D00023EFE71A4B4D
:103070001A4A1B68934206D9C02304222800217CE7
:103080009B0001F0F9F9114B6361154BDFE7002359
:103090002374EAE7CC233821AC2228009B01217459
:1030A00001F0EAF90028F2D10E4B63610E4BE38187
:1030B0000E4BCCE7F441FF1F9C61FF1FA861FF1F6F
:1030C000AA61FF1F59590000830500001541001136
:1030D000F4BC001182150000C061FF1F87130000BF
:1030E00000BD0011CD410011AAAAFFFFE8BC0011EC
:1030F000F7B5164B0192C318021D002000938823D8
:103100005B05D3181B685C1C1AD09CB2402C18D8E5
:103110008D781E0CAC466746CD782D023D43AE42FD
:1031200006D1019800280ED110000C70240A4C70B2
:1031300003249BB20733A343D218009B9A42DED3E9
:10314000FEBD4432F9E71000FAE7C046FC0F00006C
:10315000802213B503000324019189B25201073183
:103160009B18A14304305A1A88235B05C3181B68B7
:10317000591C03D190429241104016BD99B240298A
:1031800007D80B000733A343C0189042ECD30020AC
:10319000F3E74430F9E7134B134A1B68126810B584
:1031A000FA24934201D81A00F824104BE4021B6859
:1031B0009A4210D813000E4A12689A420ED3013375
:1031C00007D1F823DB029C4203D10A49054808F0E5
:1031D0009FFA200010BDFC24E402ECE7FE24E40288
:1031E000F7E7C04600C0071100D0071100E0071143
:1031F00000F00711FFFFFF7FF0B59BB015000490B2
:103200000391402A00D9A0E006AB59801A80FFF74D
:10321000C2FF0400042816D9002206A9FFF768FFA0
:10322000052810D906AB1B88AB420CD1002D07D066
:10323000514B2A000499C01808F022FB002802D143
:1032400001201BB0F0BD06AB1D8020000699FFF7E2
:103250007FFF041E7BD1069B0793FFF79CFF802313
:103260005B01C618802307001B039E4201D3F8268A
:10327000F60288235B05F31801931B68013302D023
:10328000019808F09DFB3D49019808F041FA3B1D6B
:103290000293331D05938822029B52059B181B68DD
:1032A00008935A1C3CD044219AB20091402A04D879
:1032B0000320D11D814389B2009103991B0C8B42DD
:1032C00024D0402A22D80122300008A9FFF710FF9D
:1032D000021E1BD1380008A9FFF70AFF04000428CA
:1032E00031D9009A059B9B1880225201B218934253
:1032F00040D288235B05C118009A09A808F008FC91
:103300001D4B009A09A9F01808F032FC009A029BA4
:103310009446634402931A4B029AFB189A42BAD31A
:1033200088235B05FC1821680198013908F0F0F941
:10333000200008F045FB039A07AB5A80300007993C
:10334000FFF706FF0400002C03D1002079E70428D2
:10335000FBD988235B05E018069908F0D9F9032307
:10336000EA1C9A4300D16BE7034B0499E01808F07C
:10337000FFFB65E70424ECE704000011FFFFFF7F7B
:10338000F80F0000F7B505001400402A21D80027E7
:1033900001AE71803780FFF7FEFE042816D93A008F
:1033A0003100FFF7A5FE042810D93688BC420BD0A7
:1033B000BD4209D0221CB44200D9321C064B92B245
:1033C000C118280008F0A4FB30B2FEBDC04300B213
:1033D000FBE703204042F8E70400001137B5042260
:1033E00004000D0001A81649FFF7CCFF02000428D5
:1033F0000BD1019BA34208D3AB4204D0104901A8D2
:103400000195FFF7F9FE01203EBD0E4C2368200018
:10341000019308F0D5FA019920000139019108F0D3
:1034200077F980235B01E418074B9C42EED104221C
:10343000034901A80195FFF7DFFE0020E4E7C0463D
:103440005555000000C007110000081130B589B0C3
:1034500008F0AEF810226946254808F0F1F9254B2E
:10346000009A9A420ED1019B029A0F2B33D8002169
:1034700001240698013B08D2002900D00292029B49
:10348000013331D10023029325E0551CF2D1020013
:103490002100EFE710341022200004A908F0D0F931
:1034A000029B013301D1069B0293882304995B059B
:1034B000C918059B06981A03120B049105928142C4
:1034C00003D02B4201D108F023FB019B013B019368
:1034D000019B002BDED1029B002B03D004930498A8
:1034E0004168084709B030BDE025014C2D03EFE7E6
:1034F00000000111504859368022F8B5964C974B80
:10350000D200002120001C6008F05AFB2300944ADE
:1035100088331A60934B1A786A23002A00D011333B
:10352000E3620A232365904B37221B780820A363AC
:103530008E4B2118E361102323628D4B3B25636181
:10354000C823DB00A36123008C331A602823013ACF
:10355000E26320646364CA67043A211DCA672100DC
:10356000BC310D602100C03108602100C4310B6006
:1035700021000635CC310D602100083DC8310D60B9
:103580002100D0310A602200D43210602200D832EB
:10359000136022000227E032210017604222DC3152
:1035A0000A6021001B3DE4310D602100E831086014
:1035B0002100EC310B6023000521F4331960230056
:1035C000F0331A602300183290331A6023009433CA
:1035D000186023001E3A98331A60AF23DB00236083
:1035E000644BFA262363644B644DE360644BF03113
:1035F000A3642300FF31FC33B600A16021611E608B
:10360000A5627325E5656D3D6565A56596255D4AF1
:10361000AD00E264666258606766A566002709250A
:10362000A767E566584F594D606720002567E26738
:103630003A6015279C30676007001A203860200028
:10364000A0300700212038602000A83007004C4837
:1036500038602000F830066026006427A436376002
:1036600026005F3FAC3637602600033FB036376038
:103670002600C637B436376026000027B8363760D4
:1036800038269E60424E96205E64424E5A66DE6147
:10369000414E9A645E62F53EFF3E9E621E269A6728
:1036A000354A8000DE661F675F67DD651D6618624C
:1036B000DA67BE23394A5B00E250394BD8382350D1
:1036C00004302250C4225200A350C623E4205B00E1
:1036D000E1500433334AE1503349344BD16034492B
:1036E000800019503349E938FF3819503249043005
:1036F000195032493248D16132491163324951631C
:103700001900F4310860CE20304940001160304982
:10371000195019002F48F83108602F49D1658221CE
:103720002E4A89005A501A002D490832D1671A00D2
:103730002C49B432116088212B4A89005A501A0052
:103740002A49883211602A4ADA6408F011F9012006
:1037500008F0BEF8F8BDC0460004FF1F4064FF1F1C
:10376000206FFF1F3044FF1F4A0AFF1F3A07000067
:1037700080C3C9019A020000DC0500006A1800003D
:1037800050C3000088130000F009FF1F204E000006
:103790006509FF1F68100000C409000040420F00C7
:1037A00010270000FC00FF1FC11BFF1F0000FF1FB0
:1037B000152CFF1FA52FFF1F3D2EFF1F811FFF1F71
:1037C0007126FF1F9D1FFF1F4921FF1F0D1FFF1F98
:1037D0009528FF1F7D29FF1FD918FF1FA127FF1F55
:1037E000C524FF1FD124FF1F0D1EFF1FC51EFF1F75
:1037F000851DFF1F0223F0B501245F4D5F4E2B7026
:103800005F4B91B01C705F4F039333680021200021
:10381000FB7006F0D9FD200006F0D0FC0023984292
:1038200005D0FA78552A02D0332A00D097E03360C9
:10383000042006F031FF07F063FFFFF75DFE07F09D
:10384000C7FF1F22012400214F4B10AE1A704F4BAF
:103850001C704F4B19704F4B19689143163A0A432D
:103860001A60602219689143403A0A431A6008F0CE
:103870001FF907F0DDFEC120FF21474B80001A58D9
:103880008A431A50C522920098588843BF39014391
:1038900099509858414908408021C901014380202E
:1038A00099509958C0050902090A0143995080218D
:1038B0003B48490107F0DCFF03232200394901940A
:1038C0000093394808F04CF92C22384905A808F033
:1038D0001FF905AC61782078023406F08FFCA6420F
:1038E000F8D1334C334B226803201A40A023DB026B
:1038F00013432360802322689B04134323602268C0
:103900002D4B1A4080239B03134323602B4A2C4BDF
:10391000934200D8012008F01BF807F041FE8023F5
:103920002268DB0413432360287808F0A1F8039B86
:103930001878C0B207F0CCFE07F072FF21490420CE
:1039400008F056F806F074FE00F0AAF800F0EAFD60
:1039500000F092FE00F00CFA002011B0F0BD0093D0
:103960002100184A042007F01BFF8023DB059C621E
:10397000FFF76CFD5CE7C0464A0AFF1F34F00040C9
:103980003044FF1FCC61FF1F480AFF1F490AFF1F79
:10399000680AFF1FBCF0004000E100E0FF00FFFFED
:1039A0003444FF1FB856FF1F3454FF1F10BC0011D2
:1039B00014F00040FF7FF8FFFFFF9FFF0080FF1F14
:1039C000206FFF1F3B00010870B500252549264ADE
:1039D00026484D6308CA1B051B0DED188242F9D11C
:1039E00000268022224B92058B630921214B224C19
:1039F0001E62224B1120DA67214BDA688A43DA60B3
:103A00009A6820490A409A60266007F0C1FF112099
:103A100008F0F6F8636C1C4A13406364EE24E4007B
:103A20006C431A4A200C0400642390420AD8FA22FC
:103A30003300D200904205D9154B0A21C01807F077
:103A4000E7FFC3B2134A11201372D48008F0A0F824
:103A5000114B1B78002B04D1104B1021187807F064
:103A6000EFFD70BD000005400806054080060540DA
:103A7000FF01000000F000400038004004E100E0D9
:103A80003CF00040FFDFFFFFFFFEFFFFB70B000031
:103A900030F8FFFFB461FF1FEE63FF1FEC61FF1FF3
:103AA000002210B51100112007F08AFE10BD0000A1
:103AB000F8B500230926364F364C3B62E3681120E7
:103AC000B343E36008F09CF8112007F061FF112078
:103AD00007F02EFF40232268102513432360802324
:103AE0006268DB02134363608023A26802211343F0
:103AF000A360A368284A08201340A3608023A2681B
:103B00009B0113430122A360236CAB432364236C0A
:103B10001343236480231B013B62226B1F4B1A401B
:103B20002263626B1A406263A26B1A40A263E26B6B
:103B30001340E363E3681A4A1340E36006F05EFB58
:103B40000121082006F06EFC8023164A5B00516CB0
:103B500011200B43536407F063FDFD21C720124B76
:103B6000124A89005A50A36B80002B43A363E36879
:103B70000F4A3343E3600F4B195811408022120261
:103B80000A431A50802292051A600B4B5D63F8BD00
:103B900000F000403CF00040FFFFDFFFEFFFEFFFD1
:103BA000FFFF7FFF003800400000FF1FC9390011F0
:103BB000FF00FFFF00E100E00000054030B503A872
:103BC00004880B20002C0ED14968074D08784978ED
:103BD000090201430A20A94205D1012120001980D0
:103BE000024B1B7A137030BD192A0000B461FF1F0D
:103BF000F7B5150008AA16884A680F4F147852784E
:103C0000120222430A24BA4214D10122DBB20192E9
:103C100000962A0007F05CFC041E0BD1074B1B68C2
:103C2000002B07D068782A780002104342425041A6
:103C3000013098472000FEBD022900003861FF1FB7
:103C400030B5012503790400BFB02B4211D00A49D9
:103C5000408806F0A9FF28420BD0084B01A95B8DD4
:103C60004D800B80064B00221B7A60880B7104F09C
:103C70008DF83FB030BDC0463061FF1F6840FF1F68
:103C8000B461FF1F10B50549054806F043FF042144
:103C9000044A054806F000FF10BDC0463061FF1F12
:103CA000FFFF00003CBC00116840FF1F10B5024838
:103CB00004F0EEFE10BDC046413C0011062310B5D5
:103CC000837010330371443B43712A33837144334F
:103CD000C37100230222012103720E4B0270417056
:103CE0001C8881724472197A0273C1729A78427385
:103CF000DA7882730322C2731A7902745A79427491
:103D00000C2282749A79C274DB7903751123C37013
:103D1000152010BDB461FF1F10B5142007F0B8FEC8
:103D2000124B14220021186007F04AFF002007F010
:103D300057FE012007F00CFD022007F0B1FC032024
:103D400004F04AF9042006F05FF9052003F088FB2F
:103D5000062004F055F8072001F052FA082006F07A
:103D60007BFE092001F03AF810BDC0463C61FF1F00
:103D700007F086FC012007F0D3FC07F021FC0000CF
:103D8000094B10B50400984205D0012904D1200048
:103D9000064906F0BFFE10BD0229FCD1013904F02E
:103DA00035FE0028F3D0F6E7FEFF00006261FF1F3A
:103DB00070B50D7A100004AA2C0016881022144049
:103DC000154220D1002E20D10A78022A18D14A6843
:103DD000517815780E4A09022943914205D00D4ABF
:103DE000914209D01C800A2404E014220A491A8056
:103DF00007F08EFE200070BD0C2208491A80F7E7FC
:103E00001C800124F6E70824F4E70B24F2E7C046FF
:103E1000F3FF0000F4FF0000BC42FF1F18BD0011BB
:103E200010B504000749084806F074FE074804F07E
:103E30006FFD0020E40704D50721054A054806F078
:103E40002BFE10BD6261FF1FFFFF0000813D0011CE
:103E500080BC0011AC40FF1F00B50C4BBFB01A78FE
:103E60000B4902A800F0C2FC6B4680B2D880002843
:103E700009D06A46074B01A91B889380064B002294
:103E8000188803F083FF3FB000BDC0464061FF1FAC
:103E90004161FF1F0641FF1F1042FF1F00B50C4B81
:103EA000BFB01A780B4902A801F0B6FE6B4680B28B
:103EB000D880002809D06A46074B01A95B8D938002
:103EC000064B0022188803F061FF3FB000BDC046DA
:103ED0006A61FF1F6B61FF1FAC40FF1F1042FF1F95
:103EE000F7B50E00377A1C0008AB11003D001A88A8
:103EF00020231D401F423CD13378022B3BD17368F5
:103F00001F785B781B023B431E4FBB4208D01E4FFD
:103F1000BB4214D01D4DAB4221D00A252800FEBD66
:103F2000002A2AD1142C2AD82200F06807F0F0FDCC
:103F3000174B1C70012CF1D9FFF7B0FFEEE7002AF8
:103F40001BD1202C1BD82200F06807F0E1FD114B9B
:103F500004211C70104B187807F072FBDEE7E3B207
:103F60000124009201940A00310007F0B1FA050023
:103F7000D4E70825D2E70125D0E70B25CEE70D25AC
:103F8000CCE7C046F3FF0000F4FF00000229000068
:103F90006A61FF1F4061FF1FEC61FF1F332310B5F3
:103FA000040003700A220749013007F0B1FD064BF7
:103FB0000F201B681A0AE37222731A0C1B0E62731D
:103FC000A37310BDB461FF1FDC61FF1F30B5012575
:103FD00003790400BFB02B4213D00B49408806F090
:103FE000E3FD28420DD06A46084B02A81B88938047
:103FF000FFF7D4FF6B46D8800022608801A903F048
:10400000C5FE3FB030BDC0466261FF1F0641FF1FC5
:1040100010B5024804F03CFD10BDC046CD3F001174
:1040200070B5160004AA148805AA15784A68507855
:10403000117800022A4A0843801805284BD807F057
:104040007FFB03131E29343F0720032C0BD80422C7
:10405000121BAA4200D92A0022491A8030000919ED
:1040600007F056FD002070BD0720112CFBD812224E
:10407000121BAA4200D92A001B491A80EEE707202A
:104080000E2CF0D80F22121BAA4200D92A00174981
:104090001A80E3E70720032CE5D80422121BAA426A
:1040A00000D92A0012491A80D8E70720032CDAD851
:1040B0000422121BAA4200D92A000E491A80CDE719
:1040C0000720032CCFD80422121BAA4200D92A00B1
:1040D00009491A80C2E700220A201A80C3E7C046B5
:1040E000DCD5FFFFCBBC00118861FF1FBBBC0011FA
:1040F000B6BC0011B1BC0011ACBC001110B50D2153
:10410000024A034806F0C8FC10BDC046A0BC00111E
:104110001C41FF1FF0B50024274E85B03000B4715C
:1041200000F0E2F8254D264BEA89297C9A422FD1EE
:104130000423300003AA00F057F90400300000F017
:1041400011F90123B371002C34D16B4699892B6886
:10415000C9BA4B4329891B4A1B145B1853806B4611
:10416000D9896B6849BA89B24B4369891B0C5B18C2
:104170001548191C1BB2834200DD011C0B0400D53D
:1041800000211388918001331380200005B0F0BD19
:104190000227220003AB3000009700F0F7F80E234F
:1041A0000400297C0122300000976B4400F0EEF8F7
:1041B0000443C3E71C00E8E7F441FF1F9C61FF1FB5
:1041C00083050000B461FF1F0F27000073B5234E65
:1041D000300000F089F8224D07236A463000297C20
:1041E00000F002F904003000002C33D16B461B783C
:1041F0007F2B2FD800F0B6F86B46D878F023020456
:104200001B031A406B469B8816495BBA9BB21A4344
:104210002B68000953432A891B0C9B184B806B4663
:104220005A789B7812031B011A436B68024353436D
:104230006A891B0C9B180C481A1C1BB2834200DDB8
:10424000021C130400D500220B888A8001330B80E6
:10425000200076BD00F086F80124F9E7F441FF1F45
:104260009C61FF1FB461FF1F0F27000070B5114C48
:10427000237C002B0FD0382B0ED10F4D280000F0DF
:1042800033F8CC23AC222800217C9B0100F0F4F809
:10429000280000F067F870BD084BE2899A42FAD115
:1042A000054D280000F020F800222800217C00F0B5
:1042B000C5F8EDE79C61FF1FF441FF1F8305000077
:1042C00010B5084B1A7C002A09D05B69002B06D078
:1042D0009847041E01D0FEF793FE200010BD012474
:1042E000F9E7C0469C61FF1F70B5C17905000C005D
:1042F000631E9C411A4BE402E41849000460C9B2F1
:10430000007906F0C5F8E979687949000131C9B248
:1043100006F0BEF8E8790930C0B207F009FB0023C7
:10432000E36661332360AA795B3B002A0ED02268E2
:104330009A43023B134323600A23E361073323625A
:1043400000232363A3630133E36370BD22689A43B0
:10435000022313432360462363610633A361EFE71F
:104360000050004070B5002504000368DD66C07988
:104370000930C0B207F044FC2900207906F024F887
:104380002900607906F020F870BD0000F8B51E0025
:1043900006AB1D78002304681700E366616007F030
:1043A00007F901238022E3662B0027615200013BBD
:1043B00008D207F0F5FA08200A4A1168002D03D147
:1043C0002800F8BD2261F2E7236F034203D023697E
:1043D000013D3370013613685B1A032BEED90125BA
:1043E000EEE7C0466008FF1F70B51C00002305689B
:1043F0001600EB66696007F0DBF801238022EB66AC
:1044000023005200013B08D207F0CAFA08200A4AEA
:104410001168002C03D1200070BD2A61F2E72B6FD8
:10442000034203D02B69013C3370013613685B1AD9
:10443000032BEED90124EEE76008FF1F002370B5BF
:1044400004681500E366616007F0B2F80123E366D3
:10445000256107F0A5FA8020064A80001168636B89
:10446000034205D113685B1A032BF8D9012070BDF4
:104470000020FCE76008FF1F70B51D0000230468E2
:104480001600E366616007F093F80123E366266196
:104490000F33626B1A42FCD02B0A23611023626B2C
:1044A0001A42FCD0EDB2256107F07AFA8020074A63
:1044B00080001168636B034205D113685B1A032BFC
:1044C000F8D9012070BD0020FCE7C0466008FF1F3E
:1044D00070B51E00002305681400EB66696007F0E4
:1044E00067F80123A619EB660F33B4420ED107F02B
:1044F00057FA80200A4A800011686B6B03420CD186
:1045000013685B1A032BF8D9012070BD217829614B
:10451000696B1942FCD00134E7E70020F5E7C0469B
:104520006008FF1F10B5084CE368002B08D18022FB
:10453000064B52021B689B186360054B1B68236087
:1045400007F01EFAA06010BDDC61FF1FC8F000403C
:10455000CCF0004070B5184A936A916A9942FBD139
:1045600016498A689A421FD39A1A8B60144B012607
:10457000186893B2D202D20E4343424300204C68E3
:104580001B0A1B1912029B180E4C0A684B60551C23
:10459000A3420CD8002801D04B600A600A4A13607D
:1045A00008680A4B186070BD581E821ADDE7084A79
:1045B00030009B182A00EAE700F00040DC61FF1F92
:1045C000140AFF1F40420F00C8F00040CCF000402A
:1045D000C0BDF0FF70B51F4C23793F2B01D93F239D
:1045E00023711D4B22791A701878C0B207F0C0F8F9
:1045F00018231A491A4A0B801A4913800B805380DA
:10460000A379194980200B800C21938001334B43FF
:10461000164D191C0001834200D9011C2980D1804C
:104620006379002B11D101336371237A012B01D8F7
:10463000022323726279237A0D4853430A21584397
:1046400007F0E6F90B4D286070BDA02BEDD9A02333
:10465000EAE7C046D061FF1F480AFF1F0E42FF1F56
:10466000DC43FF1F0C42FF1F0A42FF1F0842FF1FCF
:1046700071020000C061FF1FF8B514210020FEF791
:10468000ADFE114C011E114D09D10C22104BC1CBB6
:10469000C1C4280007F094FAFFF79CFFF8BD0C2274
:1046A00020000C49FEF76EFE0C2802D0084B43CBCD
:1046B00043C40C2228000849FEF764FE0C28EBD006
:1046C0000C220021E5E7C046D061FF1F9C61FF1F5F
:1046D0000CBD0011FC0C0000F50C0000F0B51D4CE9
:1046E0008022A5440400882069465201400507F055
:1046F000E7F9902212016A441300200032C832C345
:1047000016C816C38023144C144FA6689B0333436A
:10471000A3603B6007F0A4F98823A0685B05C0187C
:1047200007F04EF90025882329008022A0685B0548
:10473000C01840196944520007F01AFA8023013565
:10474000FF355B019D42EED1A6603E60044B9D4467
:10475000F0BDC046FCEFFFFF4C43FF1F9808FF1F52
:1047600004100000F0B5040087B0002825D068468A
:1047700007F01EF91B4C022806D1062269462000CC
:1047800007F07EF8002816D06946002301250F2681
:104790002F00E25C013310091030874038002F00F1
:1047A000324097403A0002434A610439062BEFD168
:1047B0006846FFF793FF07B0F0BD182269460A4824
:1047C00007F07EF96A46A300D358013305D01822BA
:1047D000FF21684607F0F4F9EAE70134062CF1D12D
:1047E000E9E7C0466509FF1F00090011F0B5002583
:1047F00004000E0085B0AA4200D186E04B1C087868
:1048000001934B788978377909021943F3783F0689
:104810001B040B431F43039720706570252800D1AC
:1048200096E033D8112813D806F0DAFE69002B0180
:104830002B012B012B01AA00B800B1002B012B0189
:104840002B012B012B012B012B012B010501250134
:10485000232800D1DEE0DB2800D034E1042A00D890
:10486000ACE01025052A05D0551F2A003800711D1F
:1048700007F04EF905223100200007F049F92A001F
:104880003900601D07F044F905353EE0562859D03F
:1048900010D8332800D19DE0552839D02628DAD108
:1048A0009F4B2900132218001D0007F089F9FEF71D
:1048B000A7FB5CE0712800D177E0722800D180E08E
:1048C000602800D18BE0DC28C5D1022A00D875E031
:1048D0007378BFB26370B378A370032A05D0033A2C
:1048E000390092B2F01CFEF787FC10223900E01C60
:1048F000FEF748FDC51C002807DA60705CE00C225A
:104900002000884907F004F90C25280005B0F0BD07
:10491000013A854D0C2A13D8002A0AD028000199A3
:1049200007F0F6F8FFF756FE0C2228007F49FEF745
:1049300063FC29000C22601C07F0EAF80D25E4E76F
:104940000C22EBE7784D7A4B2A0043CB43C2E9E7D0
:10495000013A734D0C2A11D8002A08D00199280079
:1049600007F0D6F80C2228007249FEF745FC290012
:104970001322601C07F0CCF81425C6E70C22EDE7E3
:1049800005226D49601C07F0C3F80625BDE7122219
:104990006A49601C07F0BCF81325B6E7082268498D
:1049A000601C07F0B5F80925AFE77178F02905D844
:1049B000644B188801F08CFD0225A6E7FF23637085
:1049C000FAE7614B012A03D072789A706270F3E7BC
:1049D0009B78F4E72000FFF7E1FA050095E7013A3C
:1049E000594B5A4D072A10D8002A10D0012128000F
:1049F0005970019907F08CF801F048F82900072256
:104A0000601C07F085F808257FE70722EEE7002203
:104A10005A70F3E7042A04D94D4D2F6006F0B0FF19
:104A2000A860FFF797FD0422039003A9601C07F01C
:104A30006FF8052569E7474D062A15D90622280093
:104A4000019906F01DFF00280ED0062201992800CA
:104A500007F05EF8062240492800FEF7CDFB01234F
:104A6000394A91780B43937029000622601C07F0A5
:104A70004FF8072549E7012AA0D07078FFF772FEAA
:104A80009AE7012800D0E6E6931E344F1A2B04D88B
:104A90007378002B09D100F015F9314B39001D78DE
:104AA000601C6A1E07F034F82FE7551E2A00019992
:104AB000380007F02DF82B49AAB23800FEF79CFB0E
:104AC00000F036F9E9E7DA281DD1042A00D875E7A5
:104AD000082A15D9B37972791B021343F2791204AB
:104AE0001A43337A1B0613433B603B6805223100AF
:104AF0002000039307F00CF80422601D03A950E77F
:104B0000FE236370F1E7DE2800D057E7511E012A2B
:104B100001D10025F9E6019800F09EFFF9E7C046B3
:104B20009C61FF1F18BD0011D061FF1FFC0C00002D
:104B30000CBD0011F50C0000A861FF1F8861FF1F6C
:104B40005043FF1F1042FF1FCC61FF1FAD42FF1FEC
:104B5000DC61FF1F6509FF1FADAC0000CD63FF1FC7
:104B6000CB63FF1FAEDE000070477047020010B538
:104B7000094B0A32094C92B2DA815A829881188222
:104B8000207802F00BFB0422054B012120781A70DB
:104B900006F056FD10BDC046DA42FF1F1664FF1F27
:104BA0001564FF1F013870B5042809D806F0C8FD48
:104BB000030928081200234B0221187806F040FD53
:104BC00070BD204B0821187806F07AFD00221E4B9C
:104BD0001A72F5E7802200241B4B1A4D52001A81ED
:104BE00008211A682878DC7206F062FD2100287816
:104BF00006F036FD012000F04FFE00F047FFDFE732
:104C0000104B0821187806F05BFD1048FFF756F8A6
:104C10000F4B104A9B79002093800F4A138080220B
:104C2000094B5200D8721A8100F036FE00F02EFFB8
:104C30000A4B9B78002BC3D0094A136006F0F8FD9D
:104C4000BEE7C046EC61FF1FC061FF1F1942FF1F96
:104C5000D061FF1FDC43FF1F0A42FF1FCC61FF1F13
:104C600034F0004010B501290BD1012809D1054BC2
:104C70001B78002B05D02622034B04485A72FFF7FD
:104C800075FF10BDEE63FF1FC061FF1FC409000068
:104C90000300F0B50A4D8E18B14202D152008018BF
:104CA000F0BD0C782F6824093C5D0F271C700C7830
:104CB00001313C402F683C5D5C700233ECE7C0463C
:104CC0000442FF1F0D22114B10B51A700C23104C1B
:104CD00010492370093A033B0F48637006F018FF30
:104CE0002D2301220D490E48A371FFF7D1FF0122A8
:104CF0000C49FFF7CDFF01220B49FFF7C9FF002246
:104D00000A491000FEF778FA10BDC046EA63FF1F9B
:104D1000CB63FF1FCBBC0011CD63FF1F6709FF1FD3
:104D2000D263FF1F6609FF1F6509FF1FAEDE00008B
:104D300070B5124C132220001149FEF723FB114DD0
:104D4000002817DDAB78002B14D0431C2B700923EF
:104D50006B70002300190370287829000130C0B25D
:104D600006F07EFD297822000139C9B2002005F045
:104D7000B1FD70BDFFF7A6FFEEE7C046CD63FF1F94
:104D8000AEDE0000CB63FF1F10B5114B1A78187010
:104D9000002A0ED000280BD10E4B1A78062A07D80D
:104DA0005423D340DB0703D50B4B187802F0F6F9F8
:104DB00010BD0028FCD0074B1B78012B02D0033B11
:104DC000022BF5D8044B0121187806F039FCEFE7E7
:104DD000EE63FF1F1564FF1F1664FF1F70B54A4E78
:104DE0004A4A4B493070012005F000FC00F0B2FE49
:104DF000FEF706F906F0A4FE032246494648FFF7EF
:104E000047FF2D24030004221C7044490130FFF7A2
:104E10003FFF30230470424D424C437083702E3B61
:104E2000062220004049EB87FEF7ACFA062813D093
:104E3000200006F0BDFD022809D00321200006F065
:104E40006FFE8D23E3706E3B23711933637106226D
:104E500020003549FEF7D0F9344B1B68FC335C6405
:104E6000FFF766FF0020FFF78FFF314C314A012129
:104E7000314B1278207802F053F9304A304B1278D7
:104E80000021207802F04CF901222E4B1A702E4B93
:104E9000DB78552B31D12D4B3B325A722C4B2D4A9E
:104EA000AB81EA812B826A822021307806F0A0FB58
:104EB0000120404205F05AFD0120404205F0F6FD78
:104EC000FFF71CF9FEF7DEFE00F0A4FC01204042D3
:104ED000FEF7A6FF012006F02BFCF02001F0DCFA23
:104EE0000121307806F0ACFB307802F0B3FA1A48B2
:104EF00006F0D6FCFEF7DCFD70BD6422174B5B7933
:104F000053431A000A32CBE7EC61FF1F694B0011D3
:104F1000654C00115043FF1F8861FF1FA861FF1FF0
:104F2000DA42FF1F6509FF1FADAC00004064FF1FA0
:104F30001664FF1F3842FF1F1942FF1FEA63FF1F5D
:104F4000CB63FF1FBC63FF1FCC61FF1FC061FF1F4E
:104F5000C4090000CE090000EE61FF1FD061FF1FF1
:104F6000F8B50A0020230D001A40194257D0574BBC
:104F70001B78002B50D0FFF7EDFA554B554C564E91
:104F800099686268737A8A1ADB039A4202D3616075
:104F9000FEF78EFD327A217A531EDBB2994205D19B
:104FA000FFF764F9002000F0A7FD0FE09142F9D36C
:104FB00000232372FFF784F9012000F09DFD474F85
:104FC0003800FEF77BFE390006F052FB637A002BB7
:104FD0001FD0013BDBB26372002B1AD1404BDB7850
:104FE000552B01D106F024FCE37A002B0CD00023D2
:104FF0003C4A3A4FE3721388380001331380FEF7BE
:105000005DFE390006F034FB642370795843FFF7E6
:10501000ADFD237A0133237220206840F8BD0BB226
:10502000002B0ADA304B187806F062FD002801D018
:1050300006F0E6FC80200002EFE70224214206D0C1
:10504000244B01201A72FFF79FFE2000E5E70B07B3
:105050001ED5FFF77FFA1E4B1E491F4C98684A6801
:10506000637A821ADB039A4202D34860FEF720FD7E
:10507000FFF726F9FFF7FAF8012000F03DFD00F0F8
:10508000E3FB2368DB0701D5FEF7C2FF0820C4E776
:105090001024214206D00D4B1B78002BD5D1FEF7F2
:1050A00005FED2E70124214207D0104800F06CF839
:1050B00006F096FB00F006FDC7E704240800204038
:1050C0002142ABD0FEF7C8FEBFE7C046EE63FF1F2C
:1050D000DC61FF1FC061FF1FD061FF1F1942FF1F6E
:1050E000CC61FF1FB461FF1FEC61FF1FFC41FF1F7C
:1050F000F0B51B4B1B4F1B883A8804001A4E1B4D02
:1051000085B09A420DD832889A420AD3184B1A8831
:105110002B889A4205D1174A174B12881B889A424E
:105120001BD0052001F00EFA3B8802AA13803388B9
:10513000019053802B88114D93800F4B02A91B883F
:10514000D3800F4B2A78188802F02AFF0D4B0821D4
:105150002878019A1C7006F003FC05B0F0BDC0462B
:10516000BA63FF1F0E42FF1F0C42FF1F0A42FF1FC0
:10517000B863FF1FB663FF1F0842FF1F1664FF1FBF
:105180001042FF1FB463FF1F13B50C4B1C78002C9B
:1051900011D1002801D00A4B18600A4A0A4B117835
:1051A0000A4A10780A4A01920A4A0092002205F03F
:1051B00089FA200016BD1124FBE7C0461564FF1FC5
:1051C000B063FF1F1464FF1F0464FF1F1664FF1FFA
:1051D000F063FF1FF463FF1F10B5064B12201B780E
:1051E000052B06D1044B13221988044B187801F0C3
:1051F00085FB10BD1564FF1F1042FF1F1664FF1FC3
:1052000010B500240122114B52421870104B1C7033
:10521000104B1A8002F01EF904220F4B21001A7065
:105220000E480C3206F014FC102221000C4806F047
:105230000FFC07220B4B1C600B4B1C700B4B1C70A4
:105240000B4B1A700B4B1C7010BDC0461664FF1F31
:105250001564FF1F1042FF1F1464FF1F0464FF1F2B
:10526000F463FF1FF063FF1FCA63FF1FC963FF1FC3
:105270001242FF1FC863FF1FF8B5174C06002578C0
:1052800006A814240078052D23D1B41F134FA5B20E
:105290001824BD421DD88D1FADB2BD4219D8FA25C4
:1052A0006D00AA4215D21D000D4F0A3DADB2BD42A0
:1052B0000FD80C4C26800C4C21800C4900240A800D
:1052C0000B4A1380FFF714FF0A4B0421187806F0ED
:1052D000F7F92000F8BDC0461564FF1F790C0000E7
:1052E000750C00000E42FF1F0C42FF1F0A42FF1FF9
:1052F0000842FF1F1664FF1FF0B50BB20D0089B006
:10530000002B00DB70E1A44E307806F0F1FB041EA8
:1053100050D00378A22B00D122E1D02B1AD0912BB0
:1053200045D143780E2B42D19C4B82889A423ED184
:105330009B4A83681278052A39D1032018567F28A2
:1053400035D0984B1B68002B31D05B68002B2ED0DA
:1053500098472CE08078072829D806F0F1F904282E
:10536000183F3F74A8D86378002B0CD101218C4BD7
:1053700019708D4B1A78002A5BD08C4B307801F075
:10538000CFFE002855D00722854B1A7051E0617876
:105390000029F8D1E378002B11D0854A854B12788B
:1053A000307801F0BDFE60706378002BEBD12000F7
:1053B00006F026FB80200002684009B0F0BD784B63
:1053C0001B78022BF3D00121307806F041F9002838
:1053D000EAD10121307806F033F9E5E76378002B54
:1053E000D1D16F4F032807D13B78052B02D1013370
:1053F0003B701EE00223FBE76F4B1A886F4B029352
:10540000002A0BD01B78002B03D00121307806F046
:10541000A7FA3B78062B04D1013BE9E7029B1A70FF
:10542000F7E7042B41D10121029B3078197006F077
:1054300007F95C4B1B68002BB9D01B68002BB6D05A
:10544000574A107884E76378554F002B27D10622FE
:10545000211D5B4806F05CFB62895A4B5A491A8051
:10546000A2895A4B1A80E3890B800521397058496B
:105470000A80584A1380228A574B1A80574B1B7850
:10548000012B09D11F2001F05DF8FA22920042435E
:105490000421307806F064FA0022484B75E7312B7E
:1054A00000D070E70022454B1A700323A0E70622C4
:1054B0000021434806F0CCFA0023454A042113801A
:1054C000444A30781380444A138006F0F9F80821E2
:1054D000307806F0F5F8A379083B5A425341304A38
:1054E00003331370304B1B78002B06D0334B3078CE
:1054F0001A78002A06D001F051FE0122314B5242A7
:105500001A8096E70121197006F09AF8F5E708214C
:10551000307806F0D5F86378002B00D047E72C4BA5
:105520002D4F0293E388029A04211380294B30788F
:1055300003932389039A138063893B8006F088F8DC
:10554000002800D033E7264B1B68002B00D12EE744
:10555000039902983A88098800881B68984726E7CB
:105560004379132B00D022E70389012B0AD11D4B6D
:105570001B78022B06D10821307806F0A1F8FFF73E
:105580002BFE14E7052000F0DDFF08210200307833
:1055900006F0E6F90BE7C0461664FF1F051400008D
:1055A0001564FF1FB063FF1F3842FF1F1942FF1F22
:1055B000EA63FF1FCB63FF1FEC63FF1FEE63FF1F58
:1055C000BD63FF1F1042FF1FC463FF1FC663FF1FA1
:1055D000BA63FF1FB863FF1FB663FF1FBC63FF1FE3
:1055E000AC63FF1FB463FF1F8020C001014200D0E5
:1055F000E2E6CB0731D5324B1B78002B1DD0314E64
:1056000005AC3378052B1AD1023B23702E4B2100B9
:105610001B7823722D4B1B7863722D4B187801F089
:1056200023FD002809D007202A4B30701B68002B6F
:1056300003D01B68002B00D098470120BCE60E2049
:10564000254B06221B7825492370254B1B78637058
:1056500002ABC01806F05CFAD8E702230800184035
:10566000194209D0174B1B78052B03D11D4B188805
:1056700006F046FA02209FE60424214203D0FFF7F9
:1056800037FD200098E6082308001840194200D191
:1056900093E6154B1C78012C03D0022C0DD008206A
:1056A0008AE6124B124A134913481B88128809884C
:1056B00000880094FFF7E0FDF1E7FFF78DFDEEE7CE
:1056C000EE63FF1F1564FF1F1242FF1FC863FF1F19
:1056D0001664FF1FB063FF1FCA63FF1F1342FF1F43
:1056E000C963FF1F1042FF1FB463FF1F0842FF1F63
:1056F0000A42FF1F0C42FF1F0E42FF1F10B502A8F7
:1057000004880B20002C10D14968087849780902D8
:1057100001430C48814209D1022119800A4B598862
:105720001170DB7800205BB2537010BD074C0A206B
:10573000A142FAD102211980034B998811705B793B
:10574000F0E7C0466E2A0000B461FF1F6F2A000018
:10575000F7B5150008AA16884A680F4F14785278D2
:10576000120222430A24BA4214D10122DBB201926E
:1057700000962A0005F0ACFE041E0BD1074B1B68F7
:10578000002B07D068782A7800021043424250412B
:10579000013098472000FEBD022900002864FF1F49
:1057A00030B5012503790400BFB02B4225D0144940
:1057B000408805F0F9F928420CD0124B01A95B8D05
:1057C00000220B8002234B800F4B5B888B8060880C
:1057D00002F0DCFA0D49608805F0E6F9C0070CD547
:1057E0000B4B01A91B8800220B8002234B80064B28
:1057F0009B888B80608802F0C9FA3FB030BDC046FC
:105800002064FF1F3C42FF1FB461FF1F1864FF1F8D
:105810009642FF1F10B5074C0749200005F07AF9A2
:105820002000064905F076F90721054A054805F0EC
:1058300033F910BDFFFF00002064FF1F1864FF1F35
:1058400038BD00113C42FF1F10B5024803F020F99B
:1058500010BDC046A15700110221430888400B40EB
:105860000A31084003430E20024AD17881430B439A
:10587000D3707047AD42FF1F064A1379410705D523
:1058800080210B4380011371907170477F210B4081
:10589000F8E7C046AD42FF1F054A5378002803D001
:1058A00080210B43537070477F210B40FAE7C046BD
:1058B000AD42FF1F0F21114BDA780A40DA705028F1
:1058C00010D901310A43DA702022D9780A43DA70FC
:1058D0004022D9780A43DA708022D97852420A43AA
:1058E000DA7005E03C28EFD82828F1D81428F3D83E
:1058F0000122D9780A43DA707047C046AD42FF1FD3
:10590000F8B57F23324D04006E789E43314B9842A8
:1059100005DD76232B70363B33436B70F8BD2E4B81
:10592000984203DA58232B701433F5E783B21A0038
:1059300000215F32294892B2294F297082422DD925
:10594000A9708C4203DA5B421CB220232B70053411
:1059500020B20A2106F05CF804B2FA239B009C42B4
:1059600033DB80232A785B4213432B7064212000B1
:1059700006F04EF80A2100B205F02AFE09B22A7894
:105980007B5C13432B700A21200006F041F80A21AA
:1059900000B205F01DFE09B27B5C0AE08022AA700D
:1059A000002CDADA5B421CB220232B705F23092C17
:1059B000E9DC1E430A2120006E7005F009FE09B2E1
:1059C000AA787B5C1343AB70A8E7632CCEDCEDE7D1
:1059D000AD42FF1F1B4E00001DFCFFFF2A08000008
:1059E00062BD00117F23F7B5194FCD013E79040048
:1059F0009E433E71EDB2632806DD093B33433B71A4
:105A000040231D437D71F7BD0300093304DA582399
:105A100033433B716C23F4E70E4B019300280BDA00
:105A20000423444224B23B710A21200005F0D0FD3A
:105A3000019B09B25B5CE4E70928F5DD0A2105F06A
:105A4000E7FF019B00B21B5C1E433E71ECE7C046C2
:105A5000AD42FF1F62BD0011F8B50A4F05003B784B
:105A60000E00002B0CD0084C2000FEF73DFC33004C
:105A70002A0020003978FEF72BFD2000FEF772FC8B
:105A8000F8BDC0463464FF1FB442FF1F70B50A4E14
:105A90000A4D07223100280005F0F2FE002809D047
:105AA000074C31000722280006F032F808212000B8
:105AB000FFF7D2FF70BDC046AD42FF1F2D64FF1F30
:105AC0002C64FF1F7F2210B50A4B59789143033A8B
:105AD0001A70103A0A435A7078220E219A70DA78B6
:105AE0008A43DA7006221A7130325A71FFF7CEFFFC
:105AF00010BDC046AD42FF1F10B5002824D0134C86
:105B00000A210223E05E05F083FF00B2FFF7F8FEF2
:105B10000423E05E642105F07BFF012100B2FFF762
:105B200061FF207AFFF7C6FE0320FFF795FE0020F5
:105B3000FFF7A2FE064B1878053843425841C0B221
:105B4000FFF7AAFEFFF7A2FF10BDC046B461FF1F1A
:105B50001564FF1F70B50024094D2800AC71FEF7D5
:105B6000C3FB10233E212800064AFEF7B1FCA042E9
:105B700000D13E34044B28001C70FEF7F3FB70BDCF
:105B8000B442FF1F52BD00113464FF1F0200F0B584
:105B900001270A480A4E51188B1A002B00DCF0BD71
:105BA000082415784308684038404000805B013C79
:105BB00058406D08002CF5D10132EDE7FFFF0000E1
:105BC00072BD0011F0B500250F269D4200DBF0BD2F
:105BD0004C5D070944403440A400A058013578408A
:105BE000F3E70000F0B589B06A460D000B000F27FF
:105BF000110010351C780133260024093E40167030
:105C000054700232AB42F5D12023024AFFF7DAFF8B
:105C100009B0F0BD78BD0011F0B54E780B7889B0B1
:105C200036020C00170001901E43012A61D9954BE2
:105C30009E4200D877E001339E421CD1062A17D13C
:105C4000CA788B7812021A430B791B0413434A79E2
:105C500012061A438C4B5A6100221A705A808B4AE2
:105C60005A608B4A9A608B4ADA60002009B0F0BD16
:105C700088225205EEE7884B9E423CD182498B78C0
:105C8000002B00D0F6E00C2A31D10F22A3789343E9
:105C9000E278120213432279120413436279120646
:105CA00013434B60E279A07912020243207A000488
:105CB0001043627A12060243CA60E27AA07A1202A4
:105CC000024376484A81834208D804236E4914224D
:105CD00001980B7005F01CFF1420C7E71201D218C1
:105CE00089235B059A42F0D801238B70BDE7022A15
:105CF000FAD00523EAE76A4A01239642E6D1FFF784
:105D00006BFA052F0CD9E378A2781B021343227992
:105D100012041A4363791B061343624A0393136008
:105D200005F086FDA1E7584D2B78002B9DD1AB786F
:105D3000002B00D1A0E02B8901339BB20093B3422A
:105D400000D091E0132AD4D9CF7C8B7C3F02122162
:105D500020001F43FFF71AFF874200D08EE0002E7D
:105D60003DD1E378A2781B0213432279E96812043B
:105D70001A4363791B06134303930A228B4212D101
:105D8000FF23A370E370237163716B89002B09D12A
:105D9000E37B227C1B0212041343A27B13431B09E7
:105DA00001336B8100226B89002B8ED0002A67D1D2
:105DB000686837013818000B6B690003039098423C
:105DC00005D9686105F0FCFDEB780133EB7068687C
:105DD0001022A11C381805F0CBFE2E8145E76F89F3
:105DE000009A7B1E9BB293423AD1E278A3781202CA
:105DF0001A43237905A81B04134362796C681206C1
:105E00001A43EB6800920392211D0C22049305F0C3
:105E10007FFE0120260004A940421036FFF7E2FE73
:105E2000013F012F17D1009A0B232861824200D035
:105E30004CE704221C49200005F09AFE042203A925
:105E4000686805F03DFEE968039AFF23914200D19E
:105E50003CE7F73B3AE73100FFF7C4FE1036DFE7D7
:105E60000923B742A4D831E7009BB34200D9FCE62E
:105E700007232BE7022329E7032327E7062325E748
:105E80000A2323E7FFFE0000BC42FF1F00000111B0
:105E9000FFFF00005048593601FF0000FFFF0011CE
:105EA00002FF000034F00040C842FF1F10B5034C51
:105EB0000B000122210000F06BFA10BD6D60001193
:105EC0000B8870B506000D000224162B11D92B008B
:105ED0000322094900F05CFA041E0AD1074B2A8804
:105EE0001B88191C934200D9111C300089B200F0A4
:105EF000EFFA200070BDC046996000115A64FF1F80
:105F000010B54A780400013A0B000220012A07D894
:105F10000A78002A04D005222000024900F038FA4D
:105F200010BDC046C76000110A7810B50B00040010
:105F30000220002A04D007222000024900F028FA9B
:105F400010BDC046736100110A7810B50B00040043
:105F50000220002A04D009222000024900F018FA89
:105F600010BDC046D961001110B5034C0B000B22C7
:105F7000210000F00DFA10BD0962001110B5034CAC
:105F80000B000D22210000F003FA10BD7B6200110E
:105F900010B5034C0B000F22210000F0F9F910BDE1
:105FA000D56200110A7810B50B0004000220002A07
:105FB00004D011222000024900F0EAF910BDC046C9
:105FC000E5620011002310B51322190000F0E0F97A
:105FD00010BD000010B5034C0B001722210000F08B
:105FE000D7F910BD37630011002310B5192219002D
:105FF00000F0CEF910BD000010B5034C0B001B22C1
:10600000210000F0C5F910BD71630011F7B5848956
:106010000D0006000121002C22D000238268D356F7
:106020001778002B1EDA0C2C1AD90C3CA4B21319C9
:1060300040880093230002F086FE431E9841013001
:106040007B06DB0F6B703F23013C1F40A4B228701E
:10605000AF70AC80002C07D0B3680133AB60002177
:106060000800FEBD0020EBE7AC60F8E70B7803709A
:106070004B8843704B881B0A83700B79C3700420D4
:1060800070470420022B06D10020537811781B02A0
:10609000009A0B43138070470B8803700B881B0A10
:1060A0004370022070470420009983420AD153783C
:1060B00010781B0203430B80D37890781B020343B4
:1060C00000204B807047F8B50D004B78012400216B
:1060D000461C03702B788B4201D82000F8BD6B78EA
:1060E000B01C4F1C012B10D1890069184B8802226B
:1060F00033704B88B9001B0A7370691805F068FC8F
:1061000004360434A4B2F9B2E4E7122359436B18FD
:106110005A88043132705B8810221B0A7370691828
:1061200005F056FC12361234ECE770B5049D1400ED
:106130001E00052B01D8042070BD637812781B0265
:1061400013432B80E378A2781B02134302226B8057
:106150002A71211D681D063E05F03AFCB2B22A8163
:10616000E92AE8D82800A11D0A3005F031FC0020FA
:10617000E2E7002310B50A789A4201D8900010BDDA
:106180009A008A185488013304705488DBB2240AB8
:106190004470948884709288120AC2700430EAE7CE
:1061A00010B51100029C062B04D004201022142BE1
:1061B00001D010BD022222714B7808781B020343E4
:1061C0002380CB7888781B02034363800431601DF1
:1061D00005F0FEFB0020ECE710B50C788B7804315D
:1061E0005C43E4B203702200013005F0F1FB601C57
:1061F00010BD0420022B06D10020537811781B0219
:10620000009A0B431380704710B50C000A880231C6
:1062100005F0DEFB208810BD70B504000D00049869
:106220001100012B01D8042070BD1678527812029B
:10623000324302800200F13255701470E125002CC7
:1062400000D10C35023B9AB24280AA42EBD802310F
:10625000043005F0BDFB0020E6E7042000998342EE
:106260000AD1537810781B0203430B80D3789078BF
:106270001B02034300204B80704710B50C000A88B6
:10628000023105F0A5FB208810BD000070B501218A
:106290001E000420049C0E400B4218D1CB40DDB2FE
:1062A0008D4214D90A49DBB2098899420FD32300E1
:1062B000EE331D703300580011184978165C09023E
:1062C000314301332152D9B28D42F4D8002070BD40
:1062D000D442FF1F10B50C000A88023105F078FB8C
:1062E000208810BD10B50C788B7804315C43E4B283
:1062F00003702200013005F06BFB601C10BD10B56F
:1063000011000298032B01D8042010BD1478527894
:10631000043B120222430280CA788C781202224384
:1063200042809AB28280EB2AEED80431063005F022
:106330004FFB0020E9E710B50C000B8803700B88B9
:106340001B0A43704B8883704B881B0AC3708A8872
:106350000430063105F03CFBA088043080B210BD4B
:106360000420012B03D100201378009A137070478A
:1063700010B50C000B8803700B881B0A43704A8809
:106380000230043105F024FB6088023080B210BD79
:10639000F0B589B003931E4B029242000700D05A19
:1063A000019102F020F81325061E2DD0029B012436
:1063B0000370019B002B04D0001903999847001922
:1063C00084B26B461B7A5BB2002B0FDA10213800C7
:1063D00002F01CFB1925002813D130003219E1B25C
:1063E00002F066FC051E0CD10C34A4B2042304AAEE
:1063F000380005A993800696948101F0AFFD051E33
:1064000002D0300005F0D4F9280009B0F0BDC04634
:106410005864FF1F70B505000C0000280CD0002048
:10642000814209D010222000044905F0D1FA012050
:106430002B7823736B78637370BDC046B8BD0011B1
:10644000F0B506000D0017001C0085B002291BD016
:106450000020102907D1022B07D0102B03D115E003
:106460000020102C08D005B0F0BD69463800FFF7B9
:10647000D1FF2A0069460BE069463000FFF7CAFFEA
:1064800022006946380004E0022BE9D12A003900D5
:10649000300005F025F9E6E7031CF02800D9F023C9
:1064A000032008499AB2013A0B80D31703400649EA
:1064B0009B189B100B80D30F04499B185B100B801B
:1064C0007047C046D842FF1FD642FF1FD442FF1F6D
:1064D000034B1B888B4202D3024B4000C1527047D2
:1064E000D842FF1F5864FF1F014B4000185A7047E5
:1064F0005864FF1F1722014B1A8070475864FF1F12
:1065000070B505000E2005F003FA041E13D0D02349
:10651000037000230622837007494570033005F09D
:1065200057FA064B2100DA8A62811B7E2373044BE3
:10653000187805F04DFB70BD7464FF1F6464FF1F85
:106540002843FF1F262803D8024B4000C05A70473B
:106550000148FCE7DA42FF1FFFFF000070B50600AC
:106560000C00094D1C220021280005F071FA074B90
:106570001E70074B1C7005F09BF90123002801D009
:10658000002312202B7070BD6464FF1F2843FF1F7F
:106590008564FF1F70B505000D4C0800E260A16026
:1065A00010220021656005F003FB012803D11021B2
:1065B000A06802F058FD10220021280005F0F8FA2A
:1065C000012803D11021606802F04DFD70BDC04666
:1065D0006464FF1F70B5041E05D1002903D0062294
:1065E0000D4805F0F5F90D4B1D78012D11D1002C4A
:1065F00005D102221A7005F02BF9280070BD002287
:106600001A70074B1B78FF2BF7D02000FFF778FF9D
:10661000F3E70025F1E7C0467464FF1F6464FF1FC1
:106620002843FF1F030010B5002801D1002010BD32
:1066300000780B4A002803D15988D1821B79137640
:106640001378022BF2D10023984200D10333137048
:10665000044B1B78FF2B01D0FFF752FF0120E6E728
:106660006464FF1F2843FF1F002911D000280CD0AD
:106670004B79012803D140225242134303E03F22C9
:106680001340032802D001204B7170474022F4E7E9
:106690000800FAE770B5094D0100287800280BD0F2
:1066A000074C0622200005F093F921002878FFF717
:1066B000DBFF200005F094FA70BDC0468464FF1F24
:1066C0005E64FF1F00290AD0012808D13F224B79C0
:1066D0009343C02B03D0403B5A425341981C704710
:1066E00070B5174D06002B78FF2B15D00A2005F04A
:1066F0000FF9041E10D0D0230370C83B8370114BD8
:1067000011491B784670C3700622043005F060F909
:106710002100287805F05CFA0C4B1B78012B0DD179
:106720000B4B1B68002B03D09B68002B00D09847B5
:10673000084B04211878084A04F0BAFF70BDC0461F
:106740002843FF1F8464FF1F5E64FF1F8064FF1FD8
:10675000AC64FF1FB064FF1F60EA0000014B986843
:106760007047C0466464FF1F014BDB6818687047C0
:106770006464FF1F074B10B5DA68136801331360B8
:10678000054B1878FF2803D08021C90104F058FF79
:1067900010BDC0466464FF1F2843FF1FF7B50E00FD
:1067A00002F0C8F8051E1CD00E4B06621F78002FA1
:1067B00000D10778AB791020019305F0A9F8041EE9
:1067C0000FD0D0230380C73B8370019BE91DC370AA
:1067D0000622043005F0FCF821003800E66005F0E0
:1067E000F7F9F7BD2643FF1F014B18787047C046E5
:1067F0008464FF1F054B002805D1054B1A78054B13
:10680000002A00D1014B18007047C0467464FF1F76
:106810008464FF1F5E64FF1F014B58687047C046C9
:106820006464FF1F024B1868431E9841C0B2704752
:106830008864FF1F421E03000120152A03D9FF3B75
:106840005A425341D8B27047F0B51C0000230E00E5
:1068500085B0039002920B70029A934201D30020FC
:1068600019E0E55C5A1CD2B2002DF8D002985119FB
:106870008142F4DC0233DFB2A35C18000193FFF71E
:10688000D9FF002807D0013D019A0399EBB233707C
:106890008A4202D1E01905B0F0BDDB19DBB2DBE7BB
:1068A00010B50C0002F09EF803001220002B03D05C
:1068B0002100588805F014F910BD000070B50E4D88
:1068C00084006359002B15D0186A002801D004F009
:1068D00057FF2B59586A002801D004F051FF2B595B
:1068E000986A002801D004F04BFF285904F048FFB3
:1068F00000232B5170BDC0469464FF1F1C4B70B524
:1069000004000E00150099420AD11A4B1B68002B97
:1069100001D1122070BD1B68002BFAD09847F9E70F
:10692000154B994215D1134B1B68002B0AD01B68DD
:10693000002B07D09847002804D1104B1C70104B37
:106940001D70E7E729002000FFF7AAFF0028E1D12A
:10695000F3E7080001F0EEFF0028DAD00378032007
:10696000A342D7D12900300005F0BAF8D2E7C046DB
:10697000FEFF00009064FF1FFFFF00008D64FF1FFB
:106980008C64FF1FF7B50400808801F0D3FF002559
:10699000A84203D00578A08802F008F81C4E33788E
:1069A000002B1FD0AB421DD11A4B28001978FFF7DE
:1069B00077FF002818D000233370A3790820A77828
:1069C000A688019304F0A4FF011E0DD0D02303700C
:1069D000CA3B8370019B477086808371280005F055
:1069E000F7F801E0002DE8D1A0880B4B8200D358C6
:1069F000002B01D0FFF762FF1721A088FFF768FD89
:106A0000A08801F027FDA08801F0FEFDF7BDC0467B
:106A10008D64FF1F8C64FF1F9464FF1FF0B587B067
:106A20001D000CAB1B88070001930DAB1B881420C5
:106A300002930EAB1B88160003930FAB1B880091CB
:106A4000049310AB1B88059304F062FF041E1AD058
:106A5000D0230370CB3B47708370C6700622290099
:106A60000430002D11D004F0B3FF019B210063819D
:106A7000029B0098A381039BE381049B2382059BD7
:106A8000A37405F0A5F807B0F0BD04F0E1FFECE752
:106A9000F7B5009308AB1B8807000C200D0016000B
:106AA000019304F035FF041E13D0280001F042FFCB
:106AB00000280FD00078D0232370C93BA370009B1F
:106AC00021002381019B6770A580E680638105F02A
:106AD0007FF8F7BD014B1878EDE7C0462843FF1F4C
:106AE00013B5040064890389C2888188C078009442
:106AF000FFF7CEFF13BD000010B5044C206800283E
:106B000003D004F03DFE0023236010BD9864FF1FF6
:106B1000A122F0B5818892004A43384B384F1B6858
:106B200004009B189D2292009B18827989B01A60FC
:106B30003B68002B5FD01D78324B1B68002B04D0C4
:106B40005B68002B01D000209847260008363100F2
:106B5000E079FFF7B7FD237DE0710200E078049350
:106B6000638A29000393238A0293E3890193A3880C
:106B700000933300FFF752FFE378002B0BD1E2893B
:106B8000A379A18802920196E2792800009201225D
:106B900001F0DAFEE0703B68002B20D0FFF7ACFF7D
:106BA000194D287800281AD0184B1978FFF778FE6D
:106BB000002814D02B78E67808200793A78804F0E3
:106BC000A7FE011E09D0D0230370CA3B4670837014
:106BD00087808671079804F0FBFF00232B70172134
:106BE000A088FFF775FCA08801F034FCA08801F0B4
:106BF0000BFD09B0F0BD064B9DE7C0463409FF1FF1
:106C00009864FF1FAC64FF1F8D64FF1F8C64FF1F1F
:106C10002843FF1FF8B5070008000E0001F08AFEA8
:106C2000041E18D02620FFF78DFC051E00D1257804
:106C3000062004F06DFE041E0DD00021062204F093
:106C400007FFD0232370C23B21006770A370A6808A
:106C5000E8B204F0BDFFF8BDF0B585B001930AAB12
:106C60001B78070002930BAB1B7808000D00009205
:106C7000039301F05FFE061E22D0102004F048FEB0
:106C8000041E1DD01022002104F0E2FE2620FFF792
:106C900059FC002800D13078D0232370C13BA37069
:106CA000009B21002372019B67706372029BA58089
:106CB000A372039BC0B2E3720C9BE36004F088FFF5
:106CC00005B0F0BDF7B50D00019001F033FE071ED1
:106CD00020D00E2004F01CFE041E1BD02620FFF73F
:106CE00031FC061E00D13E78D0232380C53B06220E
:106CF000A370F91DE01C04F06BFE019B2A00638168
:106D00000123DD401A401D40210022736573F0B25B
:106D100004F05EFFF7BD0000F0B585B002901000F2
:106D20000D0017000A9E039301F004FE041E31D0EB
:106D3000029B002B2ED1039B02795B0724D51223E3
:106D400013430422002E08D10B99002905D10C9978
:106D5000002902D10D9900291AD01A430D9B2271E6
:106D6000002B00D0C9E0002E00D1CFE0002D00D0D4
:106D7000CCE0606A002801D004F002FD1C21300044
:106D800004F0E6FE606205E002239A430E33D7E783
:106D900093432371654BBA00D458002C00D1AAE06C
:106DA000002E10D0236A002B03D11C2004F070FEAB
:106DB00020625E4BBA00D358186A002803D01C2208
:106DC000310004F005FE0C9B002B12D0574CBB0089
:106DD0001D596B6A002B03D1162004F059FE68621E
:106DE000BB00E358586A002803D016220C9904F01F
:106DF000EFFD0D9B002B11D04C4DBC006659B36AC2
:106E0000002B03D1142004F043FEB0622B59986A82
:106E1000002803D014220D9904F0DAFD380001F0A7
:106E200089FD051E67D0414BBA00D358002B62D0B4
:106E30001A6A3420002A00D11C389A6A002A01D02C
:106E4000143080B20B9A002A01D01C3080B25B6AE9
:106E5000002B01D0163080B204F05AFD041E4AD037
:106E60001822002104F0F4FD2620FFF76BFB0190AF
:106E7000002801D12B780193D0232370029B20009E
:106E800063700A23294EA370039BBD00A371AB5905
:106E9000A780196A1830002905D01C22A06004F0D0
:106EA00097FD200034307359996A002907D00300F8
:106EB00014221433E060029304F08AFD02980B9BC5
:106EC000002B08D003001C221C330B992061029375
:106ED00004F07EFD02987359596A002903D01622E6
:106EE000606104F075FD6B462100187904F070FEB6
:106EF0003800FFF7E3FC05B0F0BD10220D9B0D99A3
:106F00001B69A018236204F063FD2CE70B9B002B88
:106F100000D13FE7012D00D03CE7606A002801D096
:106F200004F02EFC1C210B982AE7C0469464FF1F36
:106F300010B5044C2068002803D004F021FC002385
:106F4000236010BD8864FF1F0B4B07B51A68002A29
:106F500001D100200EBD6946531C01201278073173
:106F6000FFF772FC0028F4D00278012310001840CB
:106F70001A42EED0EEE7C046A464FF1FF0B51F4FE3
:106F800001203B6887B0002B25D09B78059300F04B
:106F9000B3FB002821D00A20FFF7D4FA04000B200D
:106FA000FFF7D0FA164B05001E78731E9E413B6812
:106FB000F6B2191DD878FFF757FB3B682900DA7A3B
:106FC000043303929A7901930292009033002000D7
:106FD000059A04F085FC07B0F0BDFFF7B5FF002867
:106FE00005D00620FFF7AEFA04000720D8E70820F6
:106FF000FFF7A8FA04000920D2E7C0468864FF1F03
:107000008464FF1F70B50A4E040033780D00FF2B17
:107010000DD0042004F07CFC011E08D0D0230370A6
:10702000CE3B45708370C470307804F0D1FD70BDE4
:107030003843FF1F70B5040006200D0004F068FC03
:10704000011E0AD0D0230370CD3B8370054B4470E2
:107050001B688580187804F0BBFD002C01D0FFF779
:1070600067FF70BD8864FF1FF8B5264F06003B68B8
:107070000D001124002B05D10522234B1B78134250
:1070800002D112242000F8BD204A10241268002AE0
:10709000F8D01278002AF5D0DB0719D52B789A1E84
:1070A000012A1AD80C2004F0F3FC132438600028BD
:1070B000E8D000230A22437029000670023004F051
:1070C00087FCFFF75BFF041E0AD0FFF731FFD9E70B
:1070D00000F012FB0028E1D1E4E7002BE2D0D0E77A
:1070E0000B4B1B78032BCDD11D20FFF72BFA094B3F
:1070F00018800028C6D0084B04211878074A04F0ED
:10710000D7FABFE78864FF1F8564FF1FA464FF1FD1
:107110008464FF1F8264FF1FB064FF1F60EA0000E9
:10712000F7B50193194B14001A78052306000F00D8
:1071300012201A4221D0012920D1154B1D68002DA3
:107140001BD002201F2C18D8002C02D0019B002B32
:1071500013D0104B1F221E706E1C0021300004F053
:1071600077FC01992200300004F032FC310020004D
:107170002C70002F06D004F0D3FBFEBD064B12206E
:107180001D68DCE704F06CFBF7E7C0468564FF1F71
:10719000A464FF1F3843FF1FA064FF1FF8B50F4E04
:1071A00012243368002B17D01B780F3C834213D175
:1071B00000250B4F0221387804F082FA094B042194
:1071C00038781D8004F07CFA074B28001D80336856
:1071D0005C7004F075FB04002000F8BD8864FF1F9C
:1071E000B064FF1F9C64FF1F8264FF1F70B50128FD
:1071F00023D11B4C2388002B03D01A4A1578002D6D
:1072000007D0194B1B68002B02D01878FFF7C6FF78
:1072100070BD3B2B02D93C3B2380F9E7134E022182
:10722000307804F04DFAFA222388920002215A4362
:10723000307804F095FB2580EAE70B4B1B68002BA8
:10724000E6D00B4B1B785B07E2D5084B0221187880
:1072500004F036FA0022024B1A80FFF769FED7E7E6
:107260009C64FF1F8064FF1F8864FF1FB064FF1FC2
:107270008564FF1FF8B51E4D2868002803D004F070
:107280007FFA00232B601B4E3068002803D004F0E7
:1072900077FA00233360184F05243B78180020400C
:1072A000234221D0154800F02BFA3B78234213D01B
:1072B000202004F0EDFB2860002813D020220021BC
:1072C00004F0C6FB202004F0E3FB041E306005D070
:1072D0002022002104F0BCFB002004E0286804F018
:1072E0004FFA2C601320F8BD00F00AFAF4E7C0460C
:1072F000A464FF1FA064FF1F8564FF1F2C43FF1FB2
:1073000010B50A4C23681A1E0ED0002808D101308F
:10731000587004F0D5FA002805D02368002B02D05D
:107320000021FFF787FE0122100010BD8864FF1FB7
:10733000F7B5274E050033680191181E21D05C78FF
:10734000244F012C30D1FFF7FFFD002825D020006D
:10735000FFF7F8F80400412814D91F4B02211878D0
:107360001E4A04F0A5F91E4B3C3C1C8002223368E7
:107370005A703B78002B14D128000199FFF75AFE70
:107380000120FEBDFA2292004243002AEED0124BA9
:107390000221187804F0E4FAE8E7FFF7D3F80200D6
:1073A000F3E700233B70EBE73B78002BE8D10320A9
:1073B00004F0AEFA011E08D0D0230370CC3B457018
:1073C00083703368187804F003FCFFF7B1FDD7E74A
:1073D0008864FF1F8064FF1FB064FF1F60EA000025
:1073E0009C64FF1F10B51749838802008B4220D090
:1073F00011D815498B4217D0144900205B1899B257
:10740000012907D8926811785A425341D8B2FFF740
:10741000F9FD012010BD0E4A00209B1807229BB2E7
:107420009A424041C0B2F5E783681878FFF768FFD9
:10743000F0E7836899785A78090218781143FFF7C2
:1074400077FFE7E70A20000006200000F8DFFFFFD3
:10745000AFDFFFFF014B18707047C0463943FF1F75
:1074600010B5064C207001F041FA207804F0D0F9F4
:107470000521207800F062FD10BDC046B064FF1FFA
:107480000BB273B50D00002B00DBC4E0884B1878FD
:1074900004F02EFB041E0ED00378912B0FD0A22BEC
:1074A00000D1A1E0834B1878FF2852D0210004F0CE
:1074B0008FFB00284DD180200002684076BD4378C4
:1074C0000F2B76D013D8052B70D00E2BEAD18088E5
:1074D000794B98422BD8794B98421BD8784B9842DD
:1074E000E0D1A3681878591CFFF774F838E03E2BF8
:1074F000D8D18378032B74D06CD8012B6ED0022B9B
:10750000D0D1704B1B68002B23D05B68002B20D0A0
:1075100098471EE06C4BC0180C28C3D804F078F8CC
:107520001DC2C2150BC20B0B0B3223C23C00674BB2
:10753000C0180728B6D8664B1B68002B09D01B68FB
:10754000002B06D0200098470AE0A3681878FFF7C0
:10755000C7F8200004F054FAADE7A068FFF762F81E
:1075600000289FD0F5E7A3681B78002BF1D0554B7E
:107570001B68002BEDD01B68002BEAD0210055487A
:107580009847EDE74F4B1B68002BE2D01B68002BA0
:10759000DFD021005048F3E7504B1B68002BD8D0B8
:1075A0005B68002BD5D021004348E9E7FFF7EAF9F3
:1075B000CFE780884A4B984203D04A4B984200D08C
:1075C00070E7464B1B68002BC3D05B68002BC0D014
:1075D0002100D5E7153B012BBBD963E7FFF798FAEC
:1075E000B7E7FFF77DFAB4E73F4B1B78042B07D1D1
:1075F00000236A4613800179408800F0C5FCA8E7A3
:10760000364B1B68002BA4D05B68002BA1D0010077
:10761000364898479DE7012421420AD0294B1B6830
:10762000002B04D05B68002B01D00020984701207C
:1076300043E78B070AD5264B1B68002B04D05B68F9
:10764000002B01D020009847022036E704212800B3
:1076500008400D4200D131E7254E3388002B21D060
:10766000013B9BB23380002B1AD1FFF7DBF80028D7
:107670000AD0204B1C70164B1B68002B04D05B6893
:10768000002B01D020009847FFF7C6F8694601F0AB
:1076900001FD6846FEF7FEFF1D20FEF753FF308018
:1076A00004200AE7024B187804F00AF8F8E7C0460D
:1076B000B064FF1F3943FF1F0E20000001200000AF
:1076C00009100000A864FF1FFEDFFFFFAFDFFFFF10
:1076D000AC64FF1F0C2000000B2000009064FF1F13
:1076E0000D200000132000008564FF1FFFFF000035
:1076F0008264FF1F8064FF1F10B501F09BF910BD6D
:10770000014B18607047C046AC64FF1F0B88002017
:10771000162B01D817230420014A13807047C04656
:107720005A64FF1F00207047074A030011888142F6
:1077300007D091880020994202D1013080001018B2
:1077400070470020FAE7C046B864FF1FF0B58F7895
:1077500006000D00C5B01E2F15D1FFF7E5FF051E71
:1077600003D10024200045B0F0BD00223B003100D1
:10777000C078009200F0B2FB0400A81C00F0D2FB1D
:10778000FF23EB70EEE7264B062403931B78FF2BB9
:10779000E8D0182FE6D87B08224A013BDB00029292
:1077A0009A589446002ADDD0029AD3185B68002BC1
:1077B000D8D00878002802D14B78012B02D10624BA
:1077C000122FCFD107AFAB88697800976446AA68BB
:1077D000A047041EC6D1AB78029A5B08013BDB00D0
:1077E000D318390030005B689847041E0BD1AB7882
:1077F000042BB6D0039A310010782200009700F0D5
:107800006DFB0400AEE76A78002AABD1AA7805A91F
:107810003B88087130000A704B80FEF747FBA0E7F9
:107820003C43FF1FC8BD00111D4B37B505009842F2
:107830000BD000290AD1FFF777FF002805D119489E
:10784000FFF772FF002800D0058037BD01291AD14B
:10785000FFF76AFF041EF8D001235B420380A37880
:10786000FF2BF2D0FE2B07D00023E07814220093E8
:1078700029001E3300F032FBA01C00F053FB012353
:107880005B426380E1E70229DFD1013901F0BEF8F4
:107890000028DAD12800FFF747FF041EDFD1D4E724
:1078A000FEFF0000FFFF0000022210B5074B52420E
:1078B0001A80074801325A809A80DA8000F07EFAF6
:1078C000044801F025F8002010BDC046B864FF1F31
:1078D0004D770011297800110388F7B50400002BBB
:1078E00002D102252800FEBD4268022113782548F6
:1078F0005268FEF7A5FD00282ED0234F01253A88B7
:10790000002AEFD0802321885B0201259B1A99422F
:10791000E8DC0C2004F0BCF8061E31D03B8822883D
:107920009C4600231800019561469DB2491989B211
:10793000AA421BD8002801D062443A8000233000BC
:10794000082208C0210004F043F8104A1368002BF5
:1079500013D100251660C5E76268022113780C4830
:107960005268FEF76DFD0028C7D1BAE760681D01B7
:107970004019418101330198D6E71A001B68E6E7F8
:107980001325AFE736BE00113A43FF1FB464FF1F53
:1079900034BE0011014B18707047C0463C43FF1FB6
:1079A00014230A0010B51A40194204D001221021F4
:1079B00001F048F810BD4B06F9D40120884340007F
:1079C000F8E710B514008B0604D50122102101F050
:1079D00039F810BD08230A001A40194202D14BB2EF
:1079E000002B0FDA102101F02DF8002808D0230019
:1079F000F2331B78002BECD0F1342378012BE8D143
:107A00000020E6E703208907FAD4E2E7F0B51F007B
:107A1000184B85B01C68019002910392002C27D16D
:107A2000200005B0F0BDA5683301ED186B89019AFF
:107A3000934211D3029A93420ED8002F04D10A9B8D
:107A4000002B10D12C00EBE73B002978039A6868E3
:107A5000FEF7F6FC0028F2D10136B6B2A388B34295
:107A6000E1D82468DAE7A3680A9A5B891380E9E71A
:107A70000026F3E7B464FF1F37B50C000A88498875
:107A80000123914217D3002A15D0651D23792A00BE
:107A900002210A48FEF7D4FC102300280BD02379DA
:107AA0006188208800242A000094FFF7AFFF0A2392
:107AB000A04200D0230018003EBDC04636BE0011D3
:107AC00013B50A0008884988012388420BD800288A
:107AD00009D00024137905320094FFF797FF0A2399
:107AE000A04200D02300180016BD13B50A00088874
:107AF0004988012388420BD8002809D00024137933
:107B000005320094FFF782FF0A23A04200D0230031
:107B1000180016BDF0B58BB003904A8808880E0097
:107B20000123824255D3002853D00023012704ACFF
:107B300023700022718813000092FFF767FF051E73
:107B40003ED02078002835D12B78022B18D16770D1
:107B50006A8983000130E31880005A806968022234
:107B6000201803F035FF23780133DBB22370042B98
:107B700019D93B006889013080B2002BD9D01FE0B1
:107B800002236370122358436A89231804305A80F1
:107B900069681022201803F01BFF23780133DBB241
:107BA0002370002BE5D10C4A6B899B185A42534134
:107BB000DBB2DFE76378012BE4D12B78022BC7D04F
:107BC00022780A23002A04D021000398FEF798F9AE
:107BD000002318000BB0F0BD0100FFFF0F4BF0B504
:107BE00004001868002816D083685D89A54207D86C
:107BF0008288AE18B44203DA12019A18934201D176
:107C00000068EFE71E005F891036A74204D1002903
:107C100000D00D801800F0BD3300EFE7B464FF1F03
:107C200070B505000C0008880021FFF7D7FF03009E
:107C30000120002B04D022002800197AFFF7C1FE92
:107C400070BDF7B50C00002501902300EE331B78C2
:107C5000AB4201D800200AE06B00E65A0021300058
:107C6000E718FFF7BBFF002802D126800130FEBDD8
:107C7000017A0198FFF794FE002802D03B88238008
:107C8000F5E70135EDB2E0E710B504000888002102
:107C9000FFF7A4FF03000120002B03D02000197A76
:107CA000FFF77EFE10BD0000054B1B68002B01D1C5
:107CB000180004E09A6852898242F6D19888704789
:107CC000B464FF1FF0B50E27002687B0039302AB04
:107CD000FF183E8005001F4B40891400984207D0D2
:107CE0002B78013000976A6880B2FFF78FFE06009C
:107CF00002212B7818486A68FEF7A2FB00280FD0F3
:107D00006C892000FFF7D0FF002802D0013C041945
:107D1000A4B2039B002B00D01C80300007B0F0BD44
:107D200002212B780D486A68FEF78AFB0028E7D10C
:107D300002212B780A486A68FEF782FB002807D0E8
:107D4000002EDED03B88A342DBD17489013CDFE703
:107D50006C89DEE7FFFF000036BE001134BE001163
:107D600032BE001110B50C00FFF7DEFC030002204C
:107D7000002B0AD0002C00D023609B781720FE2B0C
:107D800003D00138FF2B00D1002010BD73B50D00CA
:107D900001A904001600FFF7E5FF172805D0002E03
:107DA00004D129002000FEF727F976BD0122102119
:107DB000200000F047FE0028F3D0F6E7014B1860E2
:107DC0007047C046C464FF1F37B56B469D1D010058
:107DD00004000222280003F09BFE2B88B02B0ED15A
:107DE0002379122B09D12300FA331B78012B06D1FA
:107DF0000121608800F0E0F801E01B2BF8D037BDCE
:107E000010B5054B0421187000F098F8FFF74CFDF1
:107E1000FEF770FB10BDC046C864FF1F0020F0B520
:107E20000BB20F0087B0834234DA274B187803F087
:107E30005FFE051E2BD00378A02B25D103AE3100A9
:107E4000FEF7E4F8041E0BD1B378DB0724D51F4BF3
:107E500006341B68002B03D0310068889847040063
:107E6000A868002801D003F0A3FC002C08D1184A10
:107E7000039B1340174A934206D0B3781B2B03D0C1
:107E80000121688800F098F8280003F0B9FD8020EF
:107E90000002784007B0F0BD0F4B1B68002B10D0DC
:107EA000310068889847041EDAD07378002BD7D148
:107EB000B27801A90A704B800C716888FDF7F6FF53
:107EC000CEE70624F1E7C046C864FF1FC064FF1F69
:107ED00000FFFF0000011200C464FF1FF7B501900E
:107EE000FC200D0017001E0003F012FD04001320FB
:107EF000002C12D0B02320002370089BF42267705E
:107F0000658026710830002B08D0190003F060FD51
:107F10002100019803F05CFE0020FEBD089903F0EB
:107F200097FDF5E710B5041E06D00078FD2803D8AC
:107F300003F016FCFF23237010BD00000A1F93B24C
:107F400010B504000220032B05D882400020024B0C
:107F5000D1529B189C7010BDE864FF1F0B8870B550
:107F6000043B04000D000220032B0BD8012120004C
:107F700000F04CFD03001420002B03D0290020004A
:107F800000F0DEFB70BD000007B51300034A00924D
:107F90000A00012100F02CFC0EBDC046C581001175
:107FA00007B5019203220092024B0A00122100F051
:107FB00049FC0EBD4382001107B56B4601AA118032
:107FC0000449D88008780633012802D1190003F04B
:107FD00067FD07BDC964FF1F0C4B10B51870002367
:107FE000FF210B4A1380138193819380094A5380A8
:107FF0001370517293819372D174D3821375517738
:1080000003F016FD00F0FCF910BDC046F864FF1F38
:10801000E864FF1FCA64FF1FF0B58DB06B460020F7
:1080200003910C229B5E834200DBB0E05D4B18782D
:1080300003F05EFD051E00D1A4E00378902B00D074
:108040009DE006AF01004688380000F013FA796819
:108050000400002900D19CE03B88052B6ED13B89B0
:10806000032B1CD905AC200000F0A2F86288172A67
:1080700061D83989131D994231D179682378043147
:108080000291D90738D5607800F08EF9071E06D026
:10809000002303712378012B08D0132B23D0A86869
:1080A000002800D178E003F083FB75E06288029934
:1080B00009A800F0A6F80290380000F08BF909AA90
:1080C0002378387A0192002231000092029A00F05F
:1080D00012F9380000F064F9029B002BDFD0300069
:1080E00000F080F9DBE70378032BD8D1628802998E
:1080F00009A800F0D6F8DEE7122B13D1029909A8DF
:1081000000F0B5F8021EEAD127498B88002BC6D0B3
:10811000887909A92378019161780091310000F0F4
:10812000EAF8BCE7002302AA93833000617809AA29
:10813000FFF72AFFB3E71D4B0993F6E7042B02D0A4
:108140009A1F012AABD8184A043B9B00995A002970
:10815000A5D0D218907831003A0000F0AEF800288F
:108160009DD13B88042B03D001213000FFF724FF71
:10817000012C04D1A868002801D003F019FB2800C5
:1081800003F03EFC8020039B0002434018000DB02A
:10819000F0BD012800D182E701213000FFF70CFF7C
:1081A000EDE7C046F864FF1FE864FF1F01001700F9
:1081B0000B7803704B784370CB788A781B0213439B
:1081C000438070470A88030002700A88120A4270CE
:1081D0000A88012A06D14A8882704A88120AC27027
:1081E0000420704702208242FBD14A8804309A70F2
:1081F0004A88120ADA708A881A718A88120A5A71B1
:10820000EFE710B50400012082420CD94B780A78C0
:108210001B0213432380834206D1CB788A781B024A
:1082200013436380002010BD022BFBD1CB788A78EA
:108230001B02134363804B790A791B021343A3800B
:10824000F0E70B8803700B881B0A43704B88837020
:108250004B881B0AC3708B8803718B881B0A437180
:10826000CB888371CB881B0AC37108207047030039
:108270000120082A14D14A780878120202431A8091
:10828000CA788878120202435A804A790879120221
:1082900002439A80CA798879120202430020DA8068
:1082A000704710B504000120022A05D100204B7848
:1082B0000A781B021343238010BDF8B50600102076
:1082C0000F00150003F024FB04000120002C0ED049
:1082D000A0230C22290023806780201D002D07D0B9
:1082E00003F076FB2100300003F072FC0020F8BDA3
:1082F00003F0AEFBF6E7F7B51E00009008AB1420C4
:1083000017001D78019103F003FB041E12D0A22375
:108310000370019B47704380099B057146710C22D5
:108320000830002B07D0190003F052FB2100009801
:1083300003F04EFCF7BD099903F08AFBF6E737B569
:10834000041E0FD04388002B0CD00025C1881323B6
:10835000007A172201950095FFF7CDFFFF23658076
:108360006372257037BD000010B50C4904004A88BF
:10837000002A09D08B89002B05D00020CB8A02224D
:10838000834201D010BD012213000A204343002084
:108390004032C854C81842800472F3E7CA64FF1F11
:1083A0000023438003707047094B00211A0010B569
:1083B0005C88002C06D01C79844203D10A234B43ED
:1083C000D01810BD01310A330329F1D10020F8E79C
:1083D000CA64FF1F10B50400407A03F0C1F9FF23FF
:1083E000637210BD7047043010B580B203F008FA14
:1083F000002803D00421494203F09AFB10BD00007D
:1084000070B50025104CA0682580A581A580A842E4
:1084100002D003F0CDF9A56000250C4C0C4B606D2B
:108420001D80230058331D70A84202D003F0C0F90C
:10843000656500256068002801D003F0B9F90135B1
:1084400008340A2DF6D170BD9065FF1F3465FF1FFB
:108450008465FF1F70B5041E09D1054D2880A881D1
:10846000A880A868002802D003F0A2F9AC6070BD13
:108470009065FF1FF0B54B8885B0019300234360E2
:108480000A7905000F00022A00D07BE0CA88032A7F
:1084900017D98B685E7819783602DC78D8790E4364
:1084A00099781B7A24021B020C43034353495BBA9D
:1084B0000B80331D93421ED1042C04D0631F022B6A
:1084C0000ED9012015E0019A4D4B1201D35A002B11
:1084D00006D00198FFF7BEFF4A4A136901331361C2
:1084E0000421B8682E812C80494203F021FB68608A
:1084F000002005B0F0BD434D042C06D0631F022BB5
:108500000FD9EB680133EB60DBE7019A3C4B1201BA
:10851000D35A002B05D00198FFF79CFF2B6901333C
:108520002B61374B30000293019B029A1B01019390
:10853000002301998C468B52130063449C80039363
:108540009E81FFF750FF039B041E986016D0042104
:10855000B868494203F0ECFAFA880100043A2000B6
:1085600003F036FA0199029AFB888A5A043B9B1859
:10857000029A8B522B6801332B60A2E7AB6901335F
:10858000AB619EE71E4B0293019B1E01029BF35AB7
:10859000002B2DD002998C19A068002828D0012A20
:1085A00026D1FA889B189BB27352A189994217D39E
:1085B0009B1AC018B96803F00BFA029BA289F35A00
:1085C000934200D07DE700222B81A3882B80A368F3
:1085D0006B60029BF2520B4A53680133536070E7A1
:1085E000084A9368013393600198FFF733FF68E707
:1085F000044A536901335361F6E7C046FA64FF1F2A
:108600009065FF1F0065FF1F70B5051E15D10B4C4F
:108610000B4B1880230058331870606D002802D06F
:1086200003F0C6F86565250050356068002801D064
:1086300003F0BEF80834AC42F7D170BD3465FF1FBB
:108640008465FF1FF0B51700A12285B09200019349
:108650004243394B06001B680C009B18D933FF338B
:108660001D78FDF741FF0430854204DD3000FDF741
:108670003BFF0430C5B2BD4207D33A0000213000B1
:10868000019B03F035F805B0F0BD2900380003F078
:108690001FFA2300C6B250331E700393019B2900BA
:1086A0006365380003F0F4F8CBB20293002B02D0DC
:1086B000039B01361E7000262300503303931B7862
:1086C000B34204D8606D002831D10020DBE7029A64
:1086D0002800002A04D0013B1000B34200D028003B
:1086E000F700E719387002F08BFF786000280ED091
:1086F0003A78019903F06CF9019A3B780136D31866
:108700000E4A0193D369F6B20133D361D4E7039BD8
:1087100018706065A74205D1084A1320D36A013357
:10872000D362B0E7606803F043F80834F2E703F07F
:108730003FF800236365C8E73409FF1F0065FF1F8A
:10874000F7B50D0007000421686803F0F1F92B89E3
:10875000040003702B891B0A43702B8883702B88BD
:108760001B0AC3702E8902250436F6B2F42E15D8E2
:108770001B4B9F4214D10C2003F0CAF81135011E87
:108780000CD0902303708E3B0371043B4380154B48
:108790008460C680187803F01BFA00252800FEBD0F
:1087A0005C237B43104AD3180093583301931B7802
:1087B000002B0FD10300320038000099FFF742FF71
:1087C000019B05001B78002BE8D13800009902F0CE
:1087D000DFFFE3E7054A0725536A01335362DDE70C
:1087E000FEFF0000F864FF1F3465FF1F0065FF1FD8
:1087F000F0B587B0009017200F0016000193FFF727
:10880000F2FD1325041E19D00C98031E02D0019905
:10881000201D9847030AE370052302AAA0700430C4
:10882000908127700098667003A993800494FFF7E5
:1088300087FF051E02D0200002F0BAFF280007B013
:10884000F0BD0000F0B587B01F000CAB1B780391A2
:10885000059301210DAB06001C78049200F0D6F8B8
:108860001425002821D02000FFF77EFD0135041ECD
:108870001BD01149059B0A7803700132D2B2131E36
:10888000C68001D101231A000B7022713000049BB5
:1088900003990097FFF7ACFF051E09D123002100C3
:1088A0000648074A093303F0CBF8280007B0F0BDAB
:1088B000002363802370F8E7FC64FF1F3F830011EF
:1088C00030750000F8B505000E00064C064F236811
:1088D000002B02D03100280098470434BC42F6D166
:1088E000F8BDC046A065FF1FB465FF1F0123064AFF
:1088F0005B425380002313715362044A1360536038
:108900009360D36013617047B465FF1FA065FF1FBC
:108910000200002310B506499C000859002801D127
:10892000625010BD0133052BF6D11320F9E7C04684
:10893000A065FF1F034A5388181A4342584140421A
:1089400010407047B465FF1FF0B585B002930AABC5
:108950001F780CAB1B88009008000E000192039357
:10896000FFF7E8FF05001120002D1BD10E48FFF78F
:10897000E1FF04001520002C14D006220B99A771EA
:10898000E01D03F025F8019B30002371029B2900B4
:108990006371009B66802370039B6562E381FFF730
:1089A00091FF280005B0F0BDFFFF000010B5FFF7F4
:1089B000C1FF04000220002C12D060880121FFF7C3
:1089C00081FF606A002801D002F0DAFE282200212F
:1089D000200003F03DF8012300205B4263802071FA
:1089E00010BD000030B5074A074C558801001378C8
:1089F0000020A54204D05B1A59424B415842104016
:108A000030BDC046B465FF1FFFFF0000084A10B527
:108A100001230C00904208D0FFF78CFF031E04D006
:108A2000037923405A1E9341DBB2180010BDC046A3
:108A3000FEFF0000024B1879431E9841C0B27047F8
:108A4000B465FF1F70B504000D001600FFF772FF3C
:108A5000002804D10D4B9C4200D0143070BD416AF7
:108A600003790520002907D012221A40102A02D1CA
:108A70000520002EF2D10F20DB06EFD5897E0C20D9
:108A8000A9428941494249420840E7E7FEFF000008
:108A9000030010B5002800D110BD0348034A4188E7
:108AA0009142F9D09847F7E7B465FF1FFFFF000038
:108AB000002330B5C45CCD5C6C40D4540133102B22
:108AC000F8D130BD0F23002210B5C45C64002243EE
:108AD000CA54C25CD209013BF7D210BD02000100AA
:108AE00010B52032103102F09BFF10BDF0B58BB0F5
:108AF0000390102005931700049102F0C9FF009025
:108B0000102002F0C5FF009B13240190002B05D01C
:108B100000280CD11324009802F032FE019B002B98
:108B200002D0180002F02CFE20000BB0F0BD102087
:108B300002F0AEFF0600102002F0AAFF1324050089
:108B4000002E00D1AEE0002819D01022002102F042
:108B50007FFF32002900039802F062FF041E0ED14D
:108B600033787F2B51D830000099FFF7ABFF009B83
:108B70001B787F2B53D801990098FFF7A3FF300093
:108B800002F0FEFD002D02D0280002F0F9FD002CBD
:108B9000C1D1102002F07CFF0600102002F078FF07
:108BA0000290002E7CD0002878D03A000F322300AB
:108BB0000125121105D00F333B4015B25A425341E3
:108BC0001BB26A1E1201002B33D0049BD2B298183C
:108BD0000099029AFFF76CFF013D1022002130003E
:108BE00002F036FFADB2049F2D017D19AF4242D095
:108BF000002C33D0300002F0C3FD029B002B00D1CB
:108C000089E7180002F0BCFD85E729003000FFF776
:108C100059FF28002549009AFFF74AFFA7E72900D6
:108C20000098FFF74FFF28002049019AFFF740FF07
:108C3000A5E70F210F4004998A18D9B28F4208D9AD
:108C4000D15C06A819540133102BF6D1029A019970
:108C5000C0E7791A48424141C901F2E739003000C2
:108C600006AAFFF725FF3200039806A902F0D8FEF6
:108C700010370400BAE7002CBCD13000029906AAD4
:108C8000FFF716FF320006A9039802F0C9FE08227A
:108C900004003100059802F09BFEABE71324A9E71E
:108CA0001324AAE7002800D06EE733E73CBE00118A
:108CB000F0B58BB00F0016000225009000283FD0C1
:108CC000002A3DD00B1DDBB21800029302F0E0FE3B
:108CD0001135041E34D0FDF747FD05003A00009918
:108CE000201D02F05DFFEBB20393E3702B0CDBB2AF
:108CF0002F0A00936370FFB22B0E2370A7700193AD
:108D0000FDF72CFD1022010006A802F049FF21000A
:108D1000029A04AB06A8FFF7E9FE051E0DD1039BDE
:108D200008223370009B04A9B370019B7770F37025
:108D3000301D02F035FFFDF71DFD200002F020FD83
:108D400028000BB0F0BDF0B58FB00D00149E03905D
:108D500004920593002A03D1022420000FB0F0BD35
:108D6000002EF9D00398FFF7E5FD1424071EF4D078
:108D70007278337812021A43B3781B041343F278E3
:108D800012061A43036A0192934201D30133E3D1DD
:108D9000002D03D03B7901249B07DED5082200215A
:108DA00006A802F055FE059B13240433DBB218001D
:108DB000029302F06DFE051ECFD0059A049904308F
:108DC00002F0EEFE04223100280002F0E9FE390034
:108DD000102210310AA802F0E3FE2900029A06AB25
:108DE0000AA8FFF783FE041E0FD1082206A908A8CF
:108DF00002F0D6FE0822311D08A802F071FC0128FD
:108E000007D101990398FDF7C9FC280002F0B8FCCE
:108E1000A3E70124F9E7000070B51C4C05002368A6
:108E2000181E10D0002D14D11A78002A0CD1981CCD
:108E3000083202F0CDFD02F02BFC0135002808D1EC
:108E400023681D70012070BD0A331800082202F04B
:108E5000BFFD2368002BF5D0122002F059FD061E3D
:108E60000DD0C123216803704570023110220230F9
:108E700002F0AEFD23683100587802F0A9FE2068A8
:108E800002F07EFC00232360DCE7C046DC65FF1FA8
:108E9000F8B504002020FDF755FB0D4EA700BB5987
:108EA0000500002B0DD000280BD0D878FF2809D161
:108EB00008492A000C55F35907480333611802F09A
:108EC000BFFDF8BD290002F05BFE0028F0D1F8E7F5
:108ED000F865FF1FE065FF1FE9A0001170B5064DA2
:108EE00084006359002B05D0D87802F039FCFF22AA
:108EF0006359DA7070BDC046F865FF1F70B5060093
:108F00008CB00C00150000213022684602F0A0FD54
:108F100031001022684602F043FE1D20210003228A
:108F2000684402F03DFE6846FFF7D8FD2D2104009D
:108F300003222800694402F033FE20000CB070BD0B
:108F4000F0B50700160097B001931CAB1D783022D6
:108F50001EAB00910AA800211C7802F079FD1022B6
:108F600039000AA802F01CFE1022002102A802F01B
:108F70006FFD0722310002A802F012FE072202ABA9
:108F80009818631E9C41019902F00AFE02AB9C7383
:108F90002B005A1E934102AAD3730021102206A867
:108FA00002F056FD06221D9907A802F0F9FD1A20CD
:108FB00002ABC01806221F9902F0F2FD10220099A0
:108FC0000EA802F0EDFD102202AB0EA908781C7865
:108FD000013A6040D2B2087001330131002AF5D164
:108FE0000AA8FFF77BFD102212A904000EA802F0C8
:108FF000EFFC102206AB0EA908781D78013A6840F4
:10900000D2B2087001330131002AF5D10AA8FFF766
:1090100065FD044310222098E4B212A902F0C0FDBD
:10902000200017B0F0BD70B50E0014008CB0010028
:10903000102268461D0002F0B3FD3100082204A88A
:1090400002F0AEFD2100082206A802F0A9FD684644
:10905000FFF744FD04001022280008A902F0A0FD3B
:1090600020000CB070BDF8B506000D0000243719C3
:10907000AC4200D3F8BD02F043FC030A3B70631C12
:10908000DBB201379D4203D90234F054E4B2EEE77B
:109090001C00EDE773B506000C000225002819D06E
:1090A000002917D0032101A8FFF7DDFF6B469A794D
:1090B0003F231A40013313436A463000937101A9DC
:1090C0002200FFF71BFF051E04D10322E01C01A9AB
:1090D00002F07EFC280076BD03785807DA08C00F3E
:1090E000D20080009B0710439B0F1843C0B270470B
:1090F00007230B40C908C9000B43037070470000E9
:1091000070B50400FFF7EAFE134DA4006359002B6D
:1091100021D0186A002801D002F032FB2B59986E3A
:10912000002801D002F02CFB2B59D86E002801D06A
:1091300002F026FB2B59186F002801D002F020FB0B
:109140002B59586F002801D002F01AFB285902F061
:1091500017FB00232B5170BDF865FF1F0E4B8000DD
:10916000C35870B50C00002B0FD09D68002D0CD09B
:109170002B78201D0B706B784B70A97CFFF7B8FF24
:109180002B7E23726B69E36070BD102200212000EA
:1091900002F05EFCF8E7C046F865FF1F014B18605F
:1091A0007047C046F465FF1F074A030080008258DD
:1091B00010B5002A06D0D088984203D1012901D1E8
:1091C000FFF79EFF10BDC046F865FF1FF0B5264EA5
:1091D00095B087000B93BB590500099112200A92A4
:1091E000002B31D0D888FFF7A5FB04001420002CF9
:1091F0002AD0280010A9FFF7B1FFBB591E781D6ABD
:10920000002E23D00895FDF7EFFA07000020FDF7A8
:10921000F1FA0790A379E61D069310AD0CA9089802
:1092200000F0E2FA0EA9280000F0D7FA0B9B0A9989
:109230000493069B09980293079B0396019300975A
:109240000EAB0CAAFFF77CFE15B0F0BDFDF7CCFA13
:1092500006903000FDF7CEFAE31DA779079310AB17
:1092600006000893DAE7C046F865FF1F30B50C4CDE
:1092700085002A59030085B00120002A0ED018006D
:109280006946FFF76BFF2B591A78D888054B002ADF
:1092900000D1054B6A46072100F0D9FB05B030BD6F
:1092A000F865FF1FDB970011E997001130B5094CF5
:1092B0008500295985B010226846253102F088FBC7
:1092C0002A591121044BD0886A4600F0C0FB05B032
:1092D00030BDC046F865FF1F8598001130B5094CB8
:1092E0008500295985B010226846353102F070FB9F
:1092F0002A591121044BD0886A4600F0A8FB05B01A
:1093000030BDC046F865FF1FC3980011F7B54D4F3B
:1093100086001020F4590D0002F0BAFBF3592062C8
:10932000186A132200286CD0033A29009C6802F0C6
:109330004FFBF3591A780192002A58D11E6A227DF8
:10934000317B944651400122019F114201D1674671
:109350001740217D914339432175377B4F40BC46EF
:1093600060460027800701D44F08174001210220E2
:109370008F40227D82433A432275377B5740BC465B
:1093800060460027400701D497080F400420227D43
:10939000BF0082433A432275627D002794466046AF
:1093A000727B42400A4201D167460F400121627D33
:1093B0008A433A436275777B5740BC466046002734
:1093C000800701D457080F400220627D7F0082434E
:1093D00017436775767B00227E40760701D4BA0872
:1093E0000A400426617D9200B1430A4362756A789F
:1093F000002A08D06278002A05D005220533DA77E2
:1094000000221000FEBD04222979114205D1A17C61
:10941000114202D10533033AF1E7019A21782C7801
:10942000002A02D10A002100140018220429E8D8D9
:10943000042CE6D805206043034A05331218525C19
:10944000DDE7C046F865FF1F4CBE001110B50A00ED
:109450001121024B00F0FBFA10BDC0461F9900110C
:109460000B0030B587B001AD2B806B4604001100B6
:10947000981D082202F0ACFA2A000B212000024BB2
:1094800000F0E5FA07B030BD4799001110B50A00A9
:109490001121024B00F0DBFA10BDC0469B99001170
:1094A00013B50B0011006A4613706B4604000622C8
:1094B000581C02F08DFA6A4608212000014B00F08A
:1094C000C6FA13BDBB99001110B50A001121024B59
:1094D00000F0BDFA10BDC0460B9A00117FB5050023
:1094E0000B4BAA00D4580800002C0FD0666F237FC6
:1094F000E28821780396266F0296E66E0196A46EA6
:109500000094FDF709FC2800FFF7FAFD7FBDC04677
:10951000F865FF1F10B51721FFF7E0FF10BD000031
:1095200070B50A000D00064B0221040000F08FFA0E
:10953000060029782000FFF7D1FF300070BDC0463B
:10954000EB98001170B586B000236A4613708368EB
:1095500004001D78681E0A2859D801A902F0F0F805
:10956000060633373B3F43474B4F5300180000F08C
:1095700042F9062312284BD000281BD16088FFF740
:10958000D9F90823002813D04279002A47D1264B65
:109590001A78072312070BD5244B1A680723002AD1
:1095A00006D01668002E03D0290001AAB047030098
:1095B0006A4613706B461B786088002B2AD1FFF730
:1095C00067FC06B070BD180000F06CF9D4E7180015
:1095D00000F087F9D0E7180000F093F9CCE7180005
:1095E00000F0ADF9C8E7180000F0C3F9C4E71800AF
:1095F00000F0F6F9C0E7180000F0F6F9BCE7180033
:1096000000F013FAB8E7180000F013FAB4E70723E4
:109610006A46137069466088FFF782FFD1E7052329
:10962000012AC5D1024BB8E78564FF1FF065FF1F13
:10963000F465FF1FF8B52C4F8600F35904000D00A8
:10964000002B40D0DA8882423DD15A78062A33D1A5
:109650001A78002A2ED0012099681A6A097D0142E1
:1096600006D0157B054203D007225A700120F8BDB1
:109670000220014204D0157B054201D00922F4E703
:109680000420014204D0127B024201D00B22ECE7FD
:10969000164B1B68002BE9D05B68002BE6D020003E
:1096A0009847BB5900215B78122BDFD12000FFF7D0
:1096B00015FFDBE70E4BECE7112A04D1002900D09F
:1096C00032252900F2E7002D08D12000FFF732F9FA
:1096D000002803D0102302791343037121002800CE
:1096E000FDF798FAC2E7C046F865FF1FF065FF1F57
:1096F000F465FF1F70B50E4E8500AB590400002BBA
:1097000013D01B78002B11D10A4B1B68002B04D0FF
:109710005B68002B01D02000984773595B78122BAF
:1097200003D100212000FFF7D9FE70BD024BECE70A
:10973000F865FF1FF465FF1FF065FF1F094B8000F0
:10974000C3581020002B0CD01A6A002A09D09B683D
:10975000002B06D0127A1B7E101C9A4200D9181CCE
:10976000C0B27047F865FF1F70B503000D0014000C
:109770000220002A30D000292ED013700B78081D4B
:1097800053704B789370FFF7A7FCE0700120022123
:109790002B7A23716B7B034063716A7B0A4013430E
:1097A000042263716E7B1640334363716E7BF6084F
:1097B000F600334363712B7B0340A371287B014088
:1097C00000200B43A371297B0A401343A3712A7B1A
:1097D000D208D2001343A37170BD10B50A00010076
:1097E0000120FFF7C1FF10BD10B50A0001000220E3
:1097F000FFF7BAFF10BD70B506000C000220002E66
:1098000030D000292ED07378201D0B70B3784B70A8
:10981000F178FFF76DFC01223579257271794B10D3
:10982000080013409340104003438810104080000C
:10983000C9080343C9000B436373B1794B10080097
:109840001340934010400343881002409200C9081F
:109850001343C9000B4321202373FCF773FE854299
:1098600001D2122070BD2220257AFCF76BFE8542C2
:10987000F7D823781820042BF4D86378012BF1D87B
:109880000020EFE7030010B50220002909D0002BCB
:1098900007D00322481C0A7019000D3202F098F814
:1098A000002010BD03000222080010B5002B06D0D6
:1098B000002904D00E32591C02F08AF80022100050
:1098C00010BD030010B50220002909D0002B07D0DD
:1098D0000422481C0A7019000C3202F079F80020AA
:1098E00010BD10B5FFF7DEFF10BD030002200029F8
:1098F00006D0002B04D0052200200A701B784B7084
:10990000704703000220002B08D0002906D05B78A6
:1099100000200B70013B082B00D918307047030062
:1099200010B50220002909D0002B07D00622481CC0
:109930000A7019000A3202F04BF8002010BD10B571
:10994000FFF7B0FF10BD02000B00022010B5002988
:109950000ED0002A0CD00721197011885970118877
:10996000090A997011180822D81C02F031F8002059
:1099700010BD03000A00022010B5002B0CD00029F6
:109980000AD099785878090201431180901CD91C9B
:10999000082202F01DF8002010BD030010B50220BF
:1099A000002909D0002B07D00822481C0A70190092
:1099B000921802F00DF8002010BD02000B000220EA
:1099C00010B500290BD0002A09D00921197011788F
:1099D00018185970511C062201F0FAFF002010BD22
:1099E00010B5FFF75FFF10BD02000B00022010B59D
:1099F000002A09D0002907D05178197011180622C1
:109A0000581C01F0E5FF002010BD030010B5022036
:109A1000002909D0002B07D00A22481C0A7019001F
:109A2000063201F0D5FF002010BD10B5FFF73AFF58
:109A300010BD02000B00022010B5002A06D000293C
:109A400004D018005178FFF753FB002010BDF0B58B
:109A500085B017001E006A460623050008009181A4
:109A60009380FEF7C0FC1324011E02900CD0380036
:109A7000B047041E05D1280001A9FEF76FFA041EA5
:109A800002D0029801F094FE2800FFF701FA2000AE
:109A900005B0F0BDF0B504008BB0019115000021B8
:109AA000102202A801F0D4FF334EA700B8590028B5
:109AB0003CD0C388A34239D10378002B36D14278F9
:109AC000062A18D102000100553235310C3006ABA0
:109AD000FFF7A9FA002829D12000FFF72FFE020086
:109AE00006A902A801F074FF200002A901F0C8FF36
:109AF00001200BB0F0BD816E002917D00B8A112A0E
:109B000028D19D420ED101981231093A01F0E8FDA9
:109B1000012807D1BB5920009D6EFFF70FFE2900D9
:109B20000200DEE732212000FFF7D8FC2000FEF71C
:109B300001FF061E1BD0416A002918D00B8AAB42D8
:109B400015D108220198123101F0CAFD01280ED169
:109B5000716A0AE09D42E9D108220198123101F0B0
:109B6000BFFD0128E2D1BB59996E8A7EB9E720007A
:109B700001F0BEFEBCE7C046F865FF1FF0B56B4DB7
:109B800087007E5985B0337802900393002B00D074
:109B900087E0B368346A01937078062817D10122F0
:109BA0001B7D134202D0217B114218D102221342A5
:109BB00002D0217B114251D10422134203D0237BD6
:109BC000134200D08BE0019B5A7DEB5991E007389E
:109BD0000428F8D801F0B4FD032E42678300B36E69
:109BE000002B03D11C2001F053FFB066EB599C6E93
:109BF000002C1CD010220021200001F029FF029827
:109C0000FFF79CFD01002000FFF72DFA01F078FE20
:109C10002082200008211230FFF725FA0298FFF772
:109C20008DFDA076EB592100D888FFF70FFC0822A4
:109C3000EB591CE0B36E002B05D01A00198AF0888E
:109C40001232FFF70DFC0222019B197DEB591142E4
:109C50003DD0207B10423AD0073208E0F488FCF770
:109C6000DBFD01002000FFF711FC0A22EB595A70BE
:109C7000029B9C002A595378073B042B11D8D088AB
:109C8000FEF758FE00284ED0C3895A08D21828493A
:109C9000029B0298CB542B5941180433254801F0FC
:109CA000CFFE05B0F0BDFCF79FFD0300012083420D
:109CB00001D100200393EB59DE88FCF79BFD03994B
:109CC00002003000FFF7ECFB019AEB59117D0422F2
:109CD00011420CD0217B114209D00B22C7E7F68834
:109CE000FCF73CFD01003000FFF7EEFB6BE7019A4B
:109CF000527D01210A4204D0607B084201D00C222F
:109D0000B5E702210A4204D0607B084201D00E224E
:109D1000ADE704210A4204D0627B0A4201D010223E
:109D2000A5E71222A3E7FA225200B0E7F865FF1F69
:109D3000FC65FF1FF3A0001110B5064B1A78042331
:109D4000100018401A4200D00348FFF727FA0020FD
:109D500010BDC0468564FF1F4043FF1F70B504005F
:109D6000FFF7D4FA051E43D12000FFF77FFA234EF8
:109D7000A400A0598268937CDB0708D50321036AFD
:109D80001B790B40012B02D1017F0B430377431D4D
:109D9000D97F8B1E022B0DD8022900D00121C0884B
:109DA000FCF790FF042133591A7F59700A431A7740
:109DB000280070BD01290CD102231022437000211C
:109DC0000C3001F045FE305910213530FFF74BF9CA
:109DD000EEE70529ECD10223D118437010220C3094
:109DE00001F0F6FD04233259117F0B431377EAE7A4
:109DF00008251828DCD1053DDAE7C046F865FF1FC5
:109E0000F0B58BB0059143887E4F9E00F459150044
:109E10000493002C15D1012902D000200BB0F0BD15
:109E2000101D57781678FFF757F9EB683200029348
:109E30002B7A0499019300903B002000FCF70CFF63
:109E4000EBE7E388049A934201D00820E6E7237801
:109E5000012B00D1D4E0059B581E092800D9CFE082
:109E600001F06EFC05CE0A29CC506C859AB229000F
:109E70000498FFF773FFD1E7200029001022453036
:109E800001F0A6FDB9594B78042B02D1013B4B7070
:109E9000C3E70B000A00253335320C310498FFF775
:109EA00095F90498FFF702FA0522431E9841BB5921
:109EB000C0005A70B2E7200029001022553001F08E
:109EC00087FD049B4F4C9D00295904980A0006AB5E
:109ED00055320C31FFF77AF929591022453106A87D
:109EE00001F0FEFB012808D10498FFF7F7F905906F
:109EF000002804D106222B595A7005988EE70823B2
:109F00000593FAE763780C2B7AD1E36E002B03D12B
:109F10001C2001F0BDFDE066BB59D86E00286FD053
:109F20001022290001F054FDBB590498DC6EFFF7A4
:109F300005FC0D22A076BB595A706EE7E06E002832
:109F40005ED063780D2B5BD12B8808220382A91C7D
:109F5000123001F03DFDBB599A68517D0222114239
:109F600026D0186A407B104222D00C32E4E7637896
:109F70000E2B45D1236F002B03D1162001F088FD55
:109F80002067BB59186F002803D01022290001F068
:109F90001FFD0F22BB59CFE763780F2B30D1206F05
:109FA0000622691C103001F013FDBB599A68517DDF
:109FB0000422114203D0196A497B1142D5D10021F4
:109FC0000498FFF78BFA28E7636F002B0DD0BB597D
:109FD000586F0028F3D01022290001F0F9FC01226B
:109FE000BB5952425B6F1A61E9E7142001F050FD42
:109FF000BB5960675B6F002BE9D126E72978DFE763
:10A0000007200BE7F865FF1F10B5064C207001F024
:10A01000EFFB06212078FDF791FF0348FEF778FC5F
:10A0200010BDC0460B66FF1FA991001100200BB2A6
:10A0300070B50D00834216DA264B187801F058FDF2
:10A04000041E0DD00378922B0ED0A02B37D0224BBC
:10A050001878FF283AD0210001F0BAFD002835D148
:10A0600080200002684070BD43780E2B0BD03E2B41
:10A07000EDD18378052B12D0082BE8D18179808827
:10A08000FFF7D8FA08E0154B82889A42DFD183683F
:10A090001878591CFEF7C0FE002817D1D7E7104BDF
:10A0A0001B785B0712D50F4B1B68002B0ED09B68EB
:10A0B000002B0BD0C289811D80889847ECE7FFF701
:10A0C00041FAA068002801D001F072FB200001F0E5
:10A0D00097FCC5E70B66FF1F3943FF1F18200000E0
:10A0E0008564FF1FF465FF1F10B50078FFF712FAB3
:10A0F00010BD10B50078FFF7FDFA10BD0C234343E7
:10A10000084A10B59B185A68002A03D0012901D1CA
:10A11000904710BD9B68002BFBD00029F9D19847D0
:10A12000F7E7C0462866FF1F01238340094A10B5A0
:10A13000946B1C439463506B98435063D46B200022
:10A140009843012901D120001843D063116B0B43C0
:10A15000136310BD00800040F0B500240127154BAB
:10A1600085B0DA6B144E03921A6C0192DA64019B8B
:10A17000E3403B4217D0039DE5403D400295E5B2E8
:10A1800002992800FFF7BAFF316A736A002908D0E4
:10A190003900002B01D0029979402800FFF7C4FF55
:10A1A00001E0002BF9D101340C36172CDFD105B0BA
:10A1B000F0BDC046008000400C66FF1F064B012129
:10A1C0005A68C2400A4204D01B68C34018000840C5
:10A1D00070471B6DF9E7C046008000400122064B26
:10A1E0008240002903D0D9680A43DA607047D968F1
:10A1F0009143D960FAE7C0460038004030B50324E7
:10A2000044430F4BE25C1B199C785D7801232D1BA6
:10A210000135AB40013BA340A140DB430C001228B9
:10A2200007D808499200521811681940214311605B
:10A2300030BD054A11680B4023431360F8E7C04660
:10A2400093BE001108F0004014F00040C21F70B52A
:10A25000D4B20623092C0BD80125084C95400029BF
:10A2600008D00021FFF7CAFF23682B432360002397
:10A27000180070BD2368AB43F8E7C04600380040C3
:10A28000214BF0B51B185B78022B21D103244443EA
:10A290001E4A1F4EA35C12199478012215008540B6
:10A2A000B76B013CE4B23D43A240B563194C1228A0
:10A2B00015D89B0000290CD117495B1899680A43EF
:10A2C0009A600123205C154A834011680B43136098
:10A2D000F0BD11495B18996891439960F1E70E4B05
:10A2E00000290DD159690A435A61225C1328E8D02C
:10A2F0000123203A93400A49086803430B60E7E7CB
:10A30000596991435961F0E70C66FF1F93BE001134
:10A3100000800040D8BE001100F00040A0F00040D6
:10A32000A4F00040F8B500241B4E1C4D1C4B1B5DD7
:10A33000012B1FD1194A9269E2401A420BD0012227
:10A34000B25693402200143AD2B2022A09D81549D3
:10A350004A6913434B61013402360C35172CE5D1A1
:10A36000F8BD0022B2560F499200521891680B4373
:10A370009360F0E7022BEED1E7B23800FFF71EFF43
:10A3800001235840C1B23800FFF77AFF3800FFF7C9
:10A3900015FF6877DFE7C04665BE00110C66FF1F3A
:10A3A0000D66FF1F00F00040012202388240054B7D
:10A3B000002903D059690A435A617047596991438A
:10A3C0005961FAE700380040F8B50E0001210F008E
:10A3D0008740114A0400D368FD43BB43D360831E0A
:10A3E0008B4201D8FFF7E0FF00212000FFF72EFF8E
:10A3F0000A4A0B4B5168012E05D139431B19516094
:10A400005E700020F8BD2940516002221C19627064
:10A410009A6915409D61F4E70038004000800040D3
:10A420000C66FF1F012210B58240074B002906D0A1
:10A4300019680A431A600121FFF7C6FF10BD1968A9
:10A4400091431960F7E7C046008000400C2370B5C7
:10A45000002543430A4A29009B181D70094B04003C
:10A460001B185D70FFF7B0FF0123A34006492800C9
:10A470000A681A430A6005490A689A430A6070BD6F
:10A480002866FF1F0C66FF1F3480004030800040AC
:10A4900070B504000E00FF2813D003250540FFF718
:10A4A000D5FF084AA3089B009B183F22ED00AA4055
:10A4B000AE40196820009143314319600121FFF734
:10A4C0008DFE70BD18380040F8B50C244443134B82
:10A4D0000500E4186368002B03D1A3681220002B49
:10A4E0001AD0022201270E4B00215B195A70280056
:10A4F0002770FFF769FF63681E1E08D0A3683E003F
:10A50000002B04D02800FFF759FE4640F6B2280081
:10A510003100FFF709FE0020F8BDC0462866FF1F86
:10A520000C66FF1FF7B5C420FF222B4B8000195883
:10A53000002491433F3A0A431A508022274F520287
:10A54000274E1A60274B1D5D002D21D0A31E012B25
:10A5500003D80121E0B2FFF727FF012D18D11F4BCF
:10A560009B69E3402B4213D0E3B218000193FFF73D
:10A5700025FE01000198FFF755FFE3B2143B022BC3
:10A580001DD801217156184A8D405369AB43536160
:10A590003B7F002B0DD0E5B22800FFF795FF280088
:10A5A000FFF70CFE7B7F0100834202D02800FFF7FB
:10A5B000A5FD01340C370236172CC3D1F7BD01219C
:10A5C00000237156F3568D40074A9B009B189A68EA
:10A5D000AA439A60DCE7C04600E100E00C66FF1F7A
:10A5E00065BE00110D66FF1F00F0004070B50E0043
:10A5F00015000400FFF72AFF0C236343094A2000DB
:10A600009B189D605E60FFF75FFFF021064B074AD5
:10A610008900051E5A5002D02000FFF717FF2800BE
:10A6200070BDC0462866FF1F0000FF1F59A1001122
:10A6300070B5134D07202C78002C1FD198222100D3
:10A640005200280001F0BCFA0123C420FF222B7025
:10A650000C4B80001C635C630B4B1C605C600B4B01
:10A66000195891433F3A0A431A50802252021A6005
:10A670000D20074A074901F0A3F8200070BDC0462D
:10A680000C66FF1F00800040A0F0004000E100E0E9
:10A6900025A5001125A30011030010B50620072BE6
:10A6A00009D8054A137001F0A3FAD7210020034B03
:10A6B000034A89005A5010BD6843FF1F0000FF1F66
:10A6C000D91AFF1F70B51D0002240C2910D8094AA1
:10A6D000CA40D2070CD5FBF741FF041E08D1059AEA
:10A6E00004992800FBF756FFFCF7C4FDFFF724FB95
:10A6F000200070BD1210000030B50D7802232C0030
:10A700009C43184201D02B431C0008252300AB4377
:10A71000284201D02B00234320241D00A5432042C2
:10A7200001D01C4325002A230D70184204D0117853
:10A730001E3B0B43137030BD0028FCD10C21137855
:10A740008B43F7E7F8B51D0006AB1B88140007AA7A
:10A750000E000B201778002B27D10A78022A49D146
:10A760004A68507811780002244A08438018042867
:10A7700040D800F0E5FF03121D1B2300F06801F034
:10A78000DFF8021CC0B2B84200D93A1CD2B2200095
:10A79000F1682A8001F01CF906E00222F3681B88A8
:10A7A0002A8023701B0A63700020F8BD0622EEE7A2
:10A7B00001232B80F3681B782370F5E7F368002BE7
:10A7C00016D008222A801A8822701A88120A62700B
:10A7D0005A88A2705A88120AE2709A8822719A885E
:10A7E000120A6271DA88A271DB881B0AE371DBE767
:10A7F0002B80D9E701202B80D7E7C04600D6FFFF8A
:10A80000F7B516000A781D0008AB1F880C0001235D
:10A81000022A18D14A685078117800022B4A08435E
:10A82000801803280FD800F08BFF02254439E06818
:10A8300001F086F8C0B20723B84204D37B19019314
:10A84000152B02DD0D231800FEBDE0682A00310043
:10A85000C01901F0BDF86B4600209B88E268D05417
:10A860001B4B1B68834203D01B68834200D0984770
:10A870000023E8E70B23002FE5D1022DE2D1737806
:10A8800032781B021343E2681380114B1B68002BC4
:10A89000EED01B68002BEBD00120E8E70B23002F44
:10A8A000D1D1062DCED12A003100E06801F090F818
:10A8B000DEE70B23002FC6D1012DC3D132787533CB
:10A8C000012AC0D8E3681A70D2E7C04600D6FFFF5D
:10A8D0001868FF1F70B50C001500072837D800F066
:10A8E0002FFF041436361B36242E182015290BD8BA
:10A8F000184E16220021300001F0AAF8220029008B
:10A90000300001F065F8002070BD18200229FBD14D
:10A910001288114B1A80F6E718200829F4D10A0092
:10A920000E48290001F0F4F8EDE718200129EBD1D9
:10A930000B4B10780B49DA69FFF7DEFEE3E71820CE
:10A940000129E1D1064B10780749DA6BF4E70220C0
:10A95000DAE7C0460068FF1FE643FF1FDC43FF1F26
:10A960006C43FF1F9443FF1FB443FF1F030010B548
:10A970000020DB0704D50721024A034800F08CF8C9
:10A9800010BDC046F0BE00116C43FF1F054A030016
:10A990001068002803D082889A4201D180687047ED
:10A9A0000068F6E7106AFF1F0A88030008009A4251
:10A9B00004D08A8804309A4200D0002070470000FA
:10A9C000F8B5F22200230D4F0D4E79680500424381
:10A9D0003370994200D07B600A4C0021200001F0C6
:10A9E00037F800231A007C60AB4202D1002033709C
:10A9F000F8BD01332280DBB2F234F5E7086BFF1FAC
:10AA0000066BFF1F146AFF1F73B56B4601900600AB
:10AA1000684615001980FCF75FFF041E11D1002D58
:10AA20000FD07689002E11D00C2001F031F80028CB
:10AA30000ED0084A0460136886808560002B02D11E
:10AA40001060200076BD1A001B68F7E70224F8E7C3
:10AA50001324F6E7106AFF1F012100220A4B10B5EC
:10AA600049420A4C198099809A719A70084B20705B
:10AA7000012019805A60FFF7A3FF2078FCF78AFFB6
:10AA80000448FDF745FF10BD2068FF1F106BFF1F36
:10AA9000086BFF1F45AB0011022310B5002802D040
:10AAA000FFF7B2FF0300180010BD0000030010B54F
:10AAB0000020DB0704D50421024A0348FFF7A4FF66
:10AAC00010BDC04604BF0011EC43FF1FF0B50E26B9
:10AAD00087B003930CAB1F8802ABF6180500080083
:10AAE00031000292FDF77AF804000120002C0FD00B
:10AAF0003088FFF74BFF03000E20002B08D05E6864
:10AB0000002E05D021002800039B029A0097B04731
:10AB100007B0F0BD0A4B10B5984207D101220023BF
:10AB200052420A808B708A808B7110BDFFF73CFF08
:10AB30000028FAD001235B42038000238370F4E7EE
:10AB4000FFFF0000F8B5050001290AD1134E0024CB
:10AB50003388F227AB4219D028001149FFF7DAFFFA
:10AB600006E0022904D10139FDF750FF0028EDD09D
:10AB7000F8BD3B0063437268D018D35A002B09D04C
:10AB80003A00002100F064FF0134E4B2054B1B7869
:10AB9000A342EED801235B423380DDE7086BFF1F41
:10ABA0002068FF1F066BFF1F10B5FFF7FDFE0300B7
:10ABB0000020834200D0987810BD0000F0B589B025
:10ABC0001C000EAB80CB03901E8810AB1B78049248
:10ABD00002930B7A0D00DB0616D42B780593022B1B
:10ABE00024D00498FFF7D2FE002812D003689C46B8
:10ABF000002B0ED0029B2200019329003B006446EB
:10AC000003980096A04705E00498FFF7BFFE0028D0
:10AC100002D10E2009B0F0BD8368002BF9D00A22C2
:10AC20002900039898470028D7D0F3E76B68587835
:10AC30001A786B4B000210439842D2D8043B9842DA
:10AC400010D2684B984242D015D8674BC0180128E3
:10AC5000C7D80B20002EDDD1EB681A7859683A80EE
:10AC6000200028E0614BC018032800D979E000F0EB
:10AC700067FD846A789E5E4B9842B2D10B20002E0D
:10AC8000C8D101233B80EB6831001B7823706889B1
:10AC9000013080B2FCF7A2FF3A88031E0ED0017883
:10ACA00002328A183A80428962704289120AA2707E
:10ACB00059680278E01C00F08BFE06E004323A800E
:10ACC00031000422601C00F0C3FE0020A2E70B202C
:10ACD000002E9FD1EB6807A91E8804233B80330A0E
:10ACE000300026706370FCF779FF051E28D004AB96
:10ACF0009A890E2304A95B183E49C668FCF7E2FF57
:10AD000000280BD12B783C486A680599FBF798FB23
:10AD1000002803D1012304AA5B42D3813278022A9E
:10AD200006D17168201D00F053FE3B8802333B8042
:10AD30000E2304AA9B181B88A3701B0AE370C4E7A8
:10AD400004ABDE81F4E70B20002E00D062E7E96857
:10AD50000398FFF729FF02233B802070000A6070F0
:10AD6000B3E70B20002E00D054E70222EB681B88CB
:10AD70003A8023701B0A6370A7E7E86800F0E0FDE3
:10AD8000C2B203000720B24200D243E70DD00299BD
:10AD9000DBB27118994202DB921BD3B20293029B81
:10ADA000E9681A003B8089195AE70023F6E70B206F
:10ADB000002E00D02EE70722EB683A801A78227026
:10ADC0005A7862705A88A2705A88120AE2701A7908
:10ADD0002271DA886271DB881B0AA37175E7C046AD
:10ADE000042900000228000000D8FFFFFFD6FFFF63
:10ADF00003280000FFFF000034BE0011F0B58DB045
:10AE00006B460020089120229B5E83423DDAA64BD0
:10AE1000187800F06DFE071E32D00378B02B2CD1CD
:10AE20000079023816281FD800F0DAFB17001E0040
:10AE30001E001E0031001E0096001E001D011E0097
:10AE400052011E0073011E00CD011E0050021E00A3
:10AE50001E001E008E021E00E302944B94491B88C4
:10AE600078880B80FBF72CF83800FCF7ADFF914B8E
:10AE70001B68002B01D038009847380000F0C0FD57
:10AE80008020089B0002434018000DB0F0BDEE2268
:10AE90000021874800F0DCFD0BAA3B7B79893889CB
:10AEA00000923A000D32FCF7B1FD0400804B1B7894
:10AEB000002C3FD146E0804B788805937F4B4100C2
:10AEC000CB5A0BAE073BDBB23288029300230193CF
:10AED0007B4B210006930093059BFFF76FFE744D9B
:10AEE000002810D1069B3A8A1B889A420BD1380061
:10AEF0000599123000F0F4FB002804D02B78628909
:10AF00009B00EB185A80162306A81B1832882000D5
:10AF10007989FCF7D7FE2B7804009A00AA1851888B
:10AF20000029C3D00133DBB22B70002807D006A95B
:10AF3000C98A9180634A12889A42BCD802E00121F2
:10AF400049429180002B04D059497888FAF7ECFFE8
:10AF50008AE73E890A2479E000253E89574B06930B
:10AF60007B88069A5B009B5A033B9D4202DB002DC7
:10AF7000F0D05BE0162206A812183B7B798900927C
:10AF80003A0030000D32FCF741FD0590002858D002
:10AF90004689017A7888FCF703FD041E44D1464BAC
:10AFA00078880793069B4100C95A454B0439C9B2BA
:10AFB00006AAD28A06930291019400930599079BF1
:10AFC000FFF7FCFD041E2FD1069B39491A88931CFC
:10AFD000002D26D14B807988384B4900CB5A511926
:10AFE000033B8B4220DD059B31485B8941190B7186
:10AFF000A91C0135C9B2EDB2059145191B0A2B7187
:10B00000059B2D490433181800F0E2FC2C4B059ADF
:10B010001B88D318DDB22C4B9E4205D00136B6B248
:10B020009CE749889942D6D0002D0CD0204C2800AE
:10B03000618800F0EDFC207021007888FAF784FF29
:10B0400012E7059CF0E7002C00D183E77B78142BF6
:10B0500000D109E716493B794E800B700C71788856
:10B06000FAF724FF00E7162406ABE418210038891C
:10B07000FCF7B4FD011E00D1B7E1788822880F4C9F
:10B0800045002C5B0A4D013CE4B2029400240F4BB6
:10B0900001940095FFF792FD041E00D014E12900F1
:10B0A0007888FAF761FFDFE6106BFF1FD842FF1FB9
:10B0B0002868FF1F1C68FF1F1C69FF1F5864FF1FC3
:10B0C0000C6AFF1FD642FF1FFFFF00002A68FF1F08
:10B0D000162406ABE41821003889FCF77FFD011E19
:10B0E00000D182E178882288AE4C45002C5BAE4DC1
:10B0F000013CE4B202947C89AC4B01940095FFF7CB
:10B100005DFD041E00D0DFE029007888FAF736FFE5
:10B11000AAE60025A44B1D803B00F6331B78A24A0B
:10B1200078880792AB4208D99E4B128806930699FD
:10B1300043005B5A013B9A4203DB0799FAF728FF69
:10B1400092E616246B00FB18059306ABE418059BEA
:10B1500021001889FCF742FD011E03D1059B012443
:10B160001E8973E77888924B2288069C09934300D6
:10B170001B5B904E013BDBB20293002300960193D0
:10B18000099BFFF71BFD041E02D0059B1E895DE78E
:10B190007B88069A5B009B5A079A1088328812189F
:10B1A000934202DC1B1A013B33807F4C0230328811
:10B1B0000999001900F00CFC2388328801359B188E
:10B1C0002380EDB2A8E70BAA3B7B798938890092EE
:10B1D0003A000D32FCF71AFC00250590059B002B68
:10B1E00004D10A24002D00D16EE060E0059B788830
:10B1F000197AFCF7D5FB0100041E63D1694C6C4B36
:10B20000788806940993069B4400E45A694B063CEF
:10B21000E4B20BAE32880793029401910093059932
:10B22000099BFFF7CBFC041E4CD1079B5E491B8892
:10B230001A1D002D30D14A80059B5B4C5A89631939
:10B240001A716B1C9BB2E318120A1A71162306A816
:10B2500032881B1879890598FCF734FDFF21AA1C58
:10B260002E1D03350B00059092B2B6B2ADB2002888
:10B2700003D006ABDB8AD9B21B0AA218651911717B
:10B280002B714C4D301D2A884949201800F0A0FB35
:10B290002B88F618B5B2A1E74988914207D17A8880
:10B2A00006995200525AEB18053A9A42C4DC3E4CB9
:10B2B0002800618800F00CFC207021007888FAF7E3
:10B2C00071FED1E5002DF2D13E89BFE6162606AB10
:10B2D000F61831003889FCF781FC3D000400FA358E
:10B2E00000282DD0037A9B060CD400227B89398953
:10B2F000788800923A000C32FFF7E8FB041E10D069
:10B300003E8915E03088FFF741FB00281AD083689A
:10B31000002B17D02100122278889847041EE4D011
:10B32000EEE72B78002B02D17888FAF74BFE002647
:10B330002B78002B00D097E5002C00D194E585E612
:10B340000124DDE70E24DBE7162506ABED18290006
:10B350003889FCF743FC041E47D0037A9B0611D4BE
:10B36000154A7B881188994203D01448814207D13D
:10B370001380134BF2261D780023D9B2A94221D3A2
:10B380000924A1E72888FFF701FB00282FD0836854
:10B39000002B2CD02100122278889847041EDFD081
:10B3A00092E7C0465864FF1F2868FF1F2A68FF1FE6
:10B3B0001C69FF1F0C6AFF1F086BFF1FFFFF0000C7
:10B3C000066BFF1F31005943546801336018615AFE
:10B3D0000029D2D13C0008342100F22200F0F8FA12
:10B3E00021007888FAF7F6FD3EE501246CE70E248B
:10B3F0006AE71D4B1A887B889A4231D07888FAF721
:10B40000F3FD31E5F223059851684343CD18C95A3D
:10B4100000291FD03B7A012B0BD16C88AB88788830
:10B42000AA1D0094FFF752FB041E02D000233B72BA
:10B430002E88F2220021280000F00AFB00232B8036
:10B44000059B0133DBB20593084B05991B78064A2F
:10B450008B42D7D801235B421380002CCED0F5E578
:10B46000002634000596EFE7086BFF1F066BFF1FF1
:10B4700070B504000E001500FFF796FA031E08D100
:10B4800031000548FFF790FA03001120002B02D08D
:10B490001C8000209D7070BDFFFF0000F8B50B4FB1
:10B4A00006003B780D001400FF2B0ED00A2000F0A0
:10B4B0002FFA011E09D0B1230380002346800371B7
:10B4C000C5800481387800F083FBF8BD2D44FF1F50
:10B4D000F7B50F0008A90600088809A90B240988F8
:10B4E000002821D10234022B1ED1557813782D0269
:10B4F0001D432B008B4301937334002B14D1FB6845
:10B50000300019000093FFF74FFB019C85420BD0E0
:10B510002A0030000099FFF7ABFF041E04D12A0077
:10B5200030007989FFF7BAFF2000FEBDF0B50E7834
:10B5300085B003900AA805880120022E0DD14C6821
:10B540002778647824023C43054FBC4205D1039818
:10B55000DBB201960095FFF7BBFF05B0F0BDC0461A
:10B5600002290000034B10B51B68002B00D0984740
:10B57000FEE7C046146BFF1F07B501A8FFF7F2FFF7
:10B58000044A05480021121A00F01AFBF8F732F9B4
:10B59000FEE7C046186BFF1F3044FF1F000000008D
:10B5A00001B40248844601BC604700BF2932FF1F36
:10B5B00001B40248844601BC604700BF75A9000081
:10B5C00001B40248844601BC604700BF85520100B7
:10B5D00001B40248844601BC604700BF350E00003C
:10B5E00001B40248844601BC604700BF413BFF1FD5
:10B5F00001B40248844601BC604700BF012400003A
:10B6000001B40248844601BC604700BF017F0000CE
:10B6100001B40248844601BC604700BF193BFF1FCC
:10B6200001B40248844601BC604700BFD92FFF1F08
:10B6300001B40248844601BC604700BFC52DFF1F0E
:10B6400001B40248844601BC604700BF0D520100AE
:10B6500001B40248844601BC604700BFC94A0100EA
:10B6600001B40248844601BC604700BF21240000A9
:10B6700001B40248844601BC604700BF056A00006F
:10B6800001B40248844601BC604700BFED4A010096
:10B6900001B40248844601BC604700BFD91B0000CA
:10B6A00001B40248844601BC604700BF2146010046
:10B6B00001B40248844601BC604700BF59520100F2
:10B6C00001B40248844601BC604700BFB352010088
:10B6D00001B40248844601BC604700BF7139FF1FB6
:10B6E00001B40248844601BC604700BFCD4C010054
:10B6F00001B40248844601BC604700BF5118FF1FD7
:10B7000001B40248844601BC604700BFC9A90000DB
:10B7100001B40248844601BC604700BF3938FF1FAE
:10B7200001B40248844601BC604700BFA54F010038
:10B7300001B40248844601BC604700BF6DBC0000F4
:10B7400001B40248844601BC604700BF2D3BFF1F87
:10B7500001B40248844601BC604700BF3D180000A8
:10B7600001B40248844601BC604700BF1147010094
:10B7700001B40248844601BC604700BFDD66010099
:10B7800001B40248844601BC604700BF014C01007F
:10B7900001B40248844601BC604700BF7D18FF1F0A
:10B7A00001B40248844601BC604700BFC56D01007A
:10B7B00001B40248844601BC604700BFD94901007A
:10B7C00001B40248844601BC604700BF6130FF1FDE
:10B7D00001B40248844601BC604700BF792DFF1FB9
:10B7E00001B40248844601BC604700BFC51D00008B
:10B7F00001B40248844601BC604700BFC92600006E
:10B8000001B40248844601BC604700BFE92800003B
:10B8100001B40248844601BC604700BF5D170000C8
:10B8200001B40248844601BC604700BFC12FFF1F1E
:10B8300001B40248844601BC604700BFED39FF1FD8
:10B8400001B40248844601BC604700BF6571010035
:10B8500001B40248844601BC604700BF291C0000B7
:10B8600001B40248844601BC604700BF5522000075
:10B8700001B40248844601BC604700BFB54C0100DA
:10B8800001B40248844601BC604700BFF30E0000CB
:10B8900001B40248844601BC604700BF090E0000A5
:10B8A00001B40248844601BC604700BF3555000022
:10B8B00001B40248844601BC604700BF5125000026
:10B8C00001B40248844601BC604700BF691F000004
:10B8D00001B40248844601BC604700BF456B0100CB
:10B8E00001B40248844601BC604700BF851F0000C8
:10B8F00001B40248844601BC604700BF091B000038
:10B9000001B40248844601BC604700BF29510100D0
:10B9100001B40248844601BC604700BF1D4D0100D0
:10B9200001B40248844601BC604700BF4D1F0000BF
:10B9300001B40248844601BC604700BF8538FF1F40
:10B9400001B40248844601BC604700BFDD520100DB
:10B9500001B40248844601BC604700BF0132FF1FAA
:10B9600001B40248844601BC604700BF8B5201000D
:10B9700001B40248844601BC604700BFADAE000080
:10B9800001B40248844601BC604700BF156B01004A
:10B9900001B40248844601BC604700BF0539FF1F5F
:10B9A00001B40248844601BC604700BF9DA9000065
:10B9B00001B40248844601BC604700BF4D38FF1FF8
:10B9C00001B40248844601BC604700BF4537FF1FF1
:10B9D00001B40248844601BC604700BFE94C010045
:10B9E00001B40248844601BC604700BFB14E00006C
:10B9F00001B40248844601BC604700BF9D35FF1F6B
:10BA000001B40248844601BC604700BF434D0100B9
:10BA100001B40248844601BC604700BF350E0000F7
:10BA200001B40248844601BC604700BFE5480000FD
:10BA300001B40248844601BC604700BF7918000089
:10BA400001B40248844601BC604700BFA94601001A
:10BA500001B40248844601BC604700BF154D010097
:10BA600001B40248844601BC604700BF9135FF1F06
:10BA700001B40248844601BC604700BFEDA5000048
:10BA800001B40248844601BC604700BF311B00007E
:10BA900001B40248844601BC604700BF3D4B010031
:10BAA00001B40248844601BC604700BFE1170000B2
:10BAB00001B40248844601BC604700BF193AFF1F29
:10BAC00001B40248844601BC604700BFC135FF1F76
:10BAD00001B40248844601BC604700BF090E000063
:10BAE00001B40248844601BC604700BF8D120000CB
:10BAF00001B40248844601BC604700BFF54E010016
:10BB000001B40248844601BC604700BF25260000FE
:10BB100001B40248844601BC604700BF810E0000AA
:10BB200001B40248844601BC604700BF055E0000C6
:10BB300001B40248844601BC604700BF554901007A
:10BB400001B40248844601BC604700BF5933FF1F5F
:10BB500001B40248844601BC604700BFF94C0100B3
:10BB600001B40248844601BC604700BF4550000054
:10BB700001B40248844601BC604700BF9136FF1FF4
:10BB800001B40248844601BC604700BF5147010030
:10BB900001B40248844601BC604700BF1930FF1F52
:10BBA00001B40248844601BC604700BF4551010012
:10BBB00001B40248844601BC604700BF1D4B010030
:10BBC00001B40248844601BC604700BFB70E0000C4
:10BBD00001B40248844601BC604700BF594F0100D0
:10BBE00001B40248844601BC604700BFC521000083
:10BBF00001B40248844601BC604700BFD91AFF1F48
:10BC000001B40248844601BC604700BFC538FF1F2D
:10BC100000030102020303030403050006020700F8
:10BC2000080209030A030B030C000D000E030F03A7
:10BC3000100311031303140315021602BD3B001178
:10BC4000F13B0011000000000200000052BC001196
:10BC5000192A0F180A000000F1590000FD24000005
:10BC600041460100198000112DA0001181740011BE
:10BC70001D7E0011F9520011FDAD0011614F001140
:10BC8000B13D0011E13E0011000000001616000059
:10BC9000020000009CBC0011F4FFF3FFD2FC000086
:10BCA000214000110000000000000000547579617F
:10BCB0000042312E340030303137006769746875C6
:10BCC000622E636F6D2F7076767800544842310093
:10BCD00002000000E4BC0011292A282A272A262A6B
:10BCE000252A242A0A180000E2040000710200003C
:10BCF00078EC0000744000001027000060F00000A5
:10BD000006640000204E0000000000000500000056
:10BD10001F501D00023CB400000117001400000079
:10BD2000A1020000303132333435363738394142E0
:10BD30004344454600000000FD56001151570011D4
:10BD4000000000000200000050BD00116F2A6E2AA2
:10BD50001A18EAD8BC80F0FC600000000000000067
:10BD600000005F066B2F363D7D077F3F777C596E65
:10BD70007971000001A00000000000006410B71DF0
:10BD8000C8206E3BAC30D9269041DC76F4516B6B09
:10BD90005861B24D3C7105502083B8ED44930FF0CB
:10BDA000E8A3D6D68CB361CBB0C2649BD4D2D38681
:10BDB00078E20AA01CF2BDBDFB349B5F80000080CE
:10BDC0000010000000000000836000110D770011DA
:10BDD000A7600011157B00112B610011EB7A001197
:10BDE000A1610011C17A0011F3610011897C001179
:10BDF0005B620011897C00118D620011437C00118F
:10BE0000A1610011797A001119620011217C0011E1
:10BE10000000000000000000FF620011217C001102
:10BE20006163001125770011052A042A012A002ADE
:10BE3000022903280128002801180018000000002A
:10BE40000000000000000000000000870101020166
:10BE500002010102010203030401030101010101C6
:10BE60000303020103000D000E0010001100130077
:10BE70001401070108010A010B011C011D02040243
:10BE800005020702080219021A021C021D0301031F
:10BE9000020317000201000504000807000B0A0056
:10BEA0001716001D1C010201010504010E0D0111F0
:10BEB00010011413011716011A19020201020B0ACC
:10BEC000020E0D02111002141302171603050403CB
:10BED0000807030B0A030E0D0001020307090A0BF2
:10BEE0000E0F101112141718191A1B1F20212200EF
:10BEF00045A7001101A80011000000000200000089
:10BF00003ABE0011000000002DB500110000000035
:08BF10000200000038BE001120
:020000041FFFDC
:1000000000000000193D001158BC001154BC001143
:100010003C61FF1F00000000000000000000000025
:1000200000000000000000000000000000000000D0
:1000300000000000000000000000000000000000C0
:1000400000000000000000000000000000000000B0
:1000500000000000000000000000000000000000A0
:100060000000000000000000000000000000000090
:100070000000000000000000000000000000000080
:100080000000000000000000000000000000000070
:100090000000000000000000000000000000000060
:1000A0000000000000000000000000000000000050
:1000B0000000000000000000000000000000000040
:1000C0000000000000000000000000000000000030
:1000D0000000000000000000000000000000000020
:1000E0000000000000000000000000000000000010
:1000F0000000000000000000000000000000000000
:1001000000000000000000000000000000000000EF
:1001100000000000000000000000000000000000DF
:1001200000000000000000000000000000000000CF
:1001300000000000000000000000000000000000BF
:1001400000000000000000000000000000000000AF
:10015000000000000000000000000000000000009F
:10016000000000000000000000000000000000008F
:10017000000000000000000000000000000000007F
:10018000000000000000000000000000000000006F
:100190004D32FF1FAD30FF1FC1660100000000009F
:1001A000000000000000000000000000000000004F
:1001B000000000000000000000000000000000003F
:1001C000000000000000000000000000000000002F
:1001D000000000000000000000000000000000001F
:1001E000000000000000000000000000000000000F
:1001F00000000000000000000000000000000000FF
:1002000000000000000000000000000000000000EE
:1002100000000000000000000000000000000000DE
:1002200000000000000000000000000000000000CE
:1002300000000000000000000000000000000000BE
:1002400000000000000000000000000000000000AE
:10025000000000000000000000000000000000009E
:10026000000000000000000000000000000000008E
:10027000000000000000000000000000000000007E
:10028000000000000000000000000000000000006E
:10029000000000000000000000000000000000005E
:1002A000000000000000000000000000000000004E
:1002B000000000000000000000000000000000003E
:1002C000000000000000000000000000000000002E
:1002D000000000000000000000000000000000001E
:1002E000000000000000000000000000000000000E
:1002F00000000000000000000000000000000000FE
:1003000000000000000000000000000000000000ED
:1003100000000000000000000000000000000000DD
:1003200000000000000000000000000000000000CD
:1003300000000000000000000000000000000000BD
:1003400000000000000000000000000000000000AD
:10035000000000000000000000000000000000009D
:10036000000000000000000000000000000000008D
:1003700079B500110000000000000000000000003E
:10038000000000000000000000000000000000006D
:10039000000000000000000000000000000000005D
:1003A000000000000000000000000000591AFF1FBC
:1003B000000000000000000000000000000000003D
:1003C000000000000000000000000000000000002D
:1003D000000000000000000000000000000000001D
:1003E000000000000000000000000000000000000D
:1003F00000000000000000000000000000000000FD
:08183800206FFF1F4118FF1F84
:10184000024981F3088802F08FF90000206FFF1F22
:1018500010B502F039FB072804D0122808D002285E
:1018600008D010BD044A0420136B01331363F8E75A
:101870000220F6E71420F4E70065FF1FF8B5070023
:101880000C0026002500503630785135002804D150
:101890000300287058342370F8BD2978CA00481E08
:1018A0008141A3183800A25C5B68C9B2FFF7D0FF82
:1018B00000280DD12B78DA00A218013350602B706C
:1018C0003378044A013B3370136A01331362D8E75B
:1018D0000123DFE70065FF1F5C234343074910B581
:1018E000C9180B0058331B78012B05D1FFF7C6FF31
:1018F000034A936A0133936210BDC0463465FF1FEB
:101900000065FF1F10B502F01FFB064A01211300FE
:1019100010CB4942D967044B136002F0D5F920007F
:1019200010BDC04600E100E01000100010B504003A
:1019300002F00AFB024B1C6002F0C6F910BDC04663
:1019400000E100E0431E5A425341A022F0B5D2010B
:101950005B421340154D164A40019B182A18127E0F
:101960008BB00191002A1BD01A000832D46F0022DC
:10197000E6B206AFE4B294420EDC2818C369002B2D
:1019800008D0019902AA117106AA049202AA16733C
:1019900003A898470BB0F0BD1978B9540132EAE7B3
:1019A0001A7D1A7806AB01261A70E6E7C067FF1F9A
:1019B00000400040F0B5254B04004001C25C85B0FA
:1019C000002A2BD01A18117E002927D0917E0029D9
:1019D00024D01179022921D11689D788D168F51B25
:1019E000ADB22A1C102D00D9102292B2BE4217D1DE
:1019F0001818012303710023C269C38003819A422E
:101A000006D06846032103730171029301A8904731
:101A10000820002C00D0192001F0FEFA05B0F0BD1E
:101A2000013C65426C41A0256442ED012C40084D0B
:101A30001B186419074D0633013A92B2AA42EDD041
:101A40001888461C1E80085C2070F5E7C067FF1FE1
:101A500000400040FFFF00000F220E4B10B59868B9
:101A6000104002380A280BD802F060F80D0A0B0A61
:101A70000A110A0A0A0A060002210020FFF762FF83
:101A800010BD0121F9E70020FFF794FFF8E7DB6FB5
:101A9000F6E7C046004000400F220E4B10B5986894
:101AA000104002380A280BD802F040F80E0A0B0A40
:101AB0000A120A0A0A0A060002210120FFF742FF61
:101AC00010BD01210800F9E70120FFF773FFF7E7D8
:101AD000DB6FF5E70090004013B5334C2378072BFC
:101AE0003DD8324B1A78324B002A39D180221968FE
:101AF00052020A431A60252001F0C4FE20232D4A19
:101B000011680B43802113606B460422C9050868E5
:101B10000733104228D080210422C905C86810422A
:101B20002ED080212020C905CA688243CA601422B1
:101B30001A701A78002A2FD18021C905C86820326E
:101B40000243CA6014221A701A78002A28D11A4B4C
:101B50001A7D22785A601D221A705932DA6013BD3C
:101B60001A6816490A40C5E7086802430A60142249
:101B70001A701A78002ACED01A78013AD2B2F7E752
:101B8000C8680243CA6014221A7019784A1ED2B279
:101B90001A700029F9D1C4E71A78013AD2B2C7E71E
:101BA0001A78013AD2B2CEE76843FF1F3044FF1FD4
:101BB0003CF000406043FF1F00200040FFFFFEFF9D
:101BC000564B70B51B68012B03D1554A936D0133F9
:101BD000936502F051F8534B534A1860534B544CE1
:101BE0001A600123534A1360534A13602378002B71
:101BF00006D006225149524802F04EF800232370C5
:101C0000504A514B10681B78C1B2002B0ED14F4C7B
:101C1000C0B223785BB2002B4FDB237824785BB211
:101C200064B21B0424021B191B1813600B1C5029DF
:101C30004ED95023464A47491078DBB2FF2202288A
:101C40004BD10868444C454D267890432A789642FB
:101C500054D9227824782E78023B5D10A31B6B4365
:101C60005201D31A10335B111843086002F0BCF91B
:101C7000031F012B45D83A4B1B78002B06D0394B5C
:101C80001B78002B02D0002002F09EF8A122364BD8
:101C900092009978354B4A431B689B188322920027
:101CA0009B181B78033B012B03D8AF20400002F0A8
:101CB0005BF901222E4BDA8270BD237824785BB267
:101CC00064B2FF33FF341B0424021B190138ABE755
:101CD000CAB2022AAED20223ACE70868254C264DD0
:101CE000267890432A78964208D9227824782D784D
:101CF000023B5B10641B63435201B2E72378DBB203
:101D0000B2E70228D5D11D4B1B78013B022B03D92A
:101D10001B4B1B78022BCCD16C20C8E79809FF1F06
:101D2000FC0FFF1F3864FF1FFF3F0000141003402B
:101D30003C64FF1F0C10034000100340D50BFF1F35
:101D40007211FF1FB40003408C09FF1F680AFF1FB8
:101D5000490AFF1F94000340460AFF1F470AFF1F5E
:101D6000F908FF1F2209FF1F300DFF1F3409FF1F55
:101D7000BC0BFF1F440AFF1F450AFF1F1C09FF1F62
:101D80002309FF1F10B502F0C7F80022014B1A808B
:101D900010BDC0463664FF1F10B502F00DF9A12139
:101DA000054A89009478054A61431268044B521829
:101DB000528C1A8010BDC046300DFF1F3409FF1F22
:101DC0003664FF1F10B50D4B0D4A9978A1239B0077
:101DD0004B431268D218531DD97F0A4B1B88994276
:101DE00009D2441C07D0C82805D0D2695B1A5A43CF
:101DF000054B5343C01802F0EFF810BD300DFF1F24
:101E00003409FF1F3664FF1F7102000070B5244DB6
:101E10002B68002B28D002F047F82B68D8402B689D
:101E20000400002B27D001F0C7FF2B68D8401D4BC2
:101E30001D4A9978A1239B004B431268D118D25CAC
:101E400091239B00002A20D0CA580132CA50174B58
:101E500017491B680868834214D3D23B181A012A19
:101E60001AD0144B186070BD02F01EF8124B19689E
:101E700001F0A2FED3E701F09FFF0F4B196801F0BC
:101E80009BFED4E70D495B18E8E7CA500C4B1B6872
:101E9000DB68E418201AE4E7F530FF30E1E7C046DC
:101EA0001C08FF1F300DFF1F3409FF1F9C09FF1F77
:101EB0003864FF1FA009FF1F1808FF1F2DFF3F00F8
:101EC0004064FF1F70B504000D00282916D10300DF
:101ED000A433C2881B889B1A0B4A9BB293420DD92C
:101EE00006006A3605223100653002F0ADF80028A0
:101EF00004D13100200001F0CFFF70BD2900200087
:101F000002F042F8F9E7C046FE7F0000F8B5050090
:101F1000012001F091FF134CA36AA26A9342FBD106
:101F2000114E336001F080FF104903000860104833
:101F3000426894460F4A17680022BC4501D24268A5
:101F4000BA1A0D4802603268AD18A422E562606AD0
:101F5000520302436262094A1278002A01D00F3B01
:101F60000B60F8BD00F00040340AFF1FE408FF1FBB
:101F700028100040180AFF1F1C0AFF1F1C09FF1F22
:101F800070B580241025E405A3682B43A36001F0FD
:101F90000BFFA368AB43A36070BD0000F7B516004C
:101FA00080221C001023D2050191916805000B438B
:101FB000936000225A4BD7301A6001F055FE9D23E2
:101FC0002A002F009B00EB58CA3201210092FC37F7
:101FD000002B01D00021009A386801F08DFF290004
:101FE000009BCB311A784F4BD3351A604B780A7867
:101FF0001B0213438A7812041A43CB781B0613433F
:10200000494A1BBA13604B790A791B0213438A7938
:1020100012041A43CB7931001B061343434A1BBAFF
:1020200013606B782A781B021343AA7812041A43B0
:10203000EB781B0613433E4A1BBA1360019A330226
:1020400013433C4A13603C4B22001B1B9C46032954
:102050003DDCB3089A0013005142B21A032A46D15C
:10206000354AE018511A827840781204000202437F
:10207000E05C043302430A600022FF2B4BDDF022B8
:102080002E4B12011A600F222D4B1A602D4A136835
:10209000002BFCD00023224A27491360091B321D64
:1020A0000B191B68043A180A23706070180C1B0E79
:1020B000A070E3700434002AF2DC802210213B6817
:1020C000D20501333B6093688B439360F7BD634651
:1020D000D578981893782D061B042B43157804396E
:1020E0002B43557804322D022B430360AFE7022ABD
:1020F0000AD1114AE05C511AE218527812020243E6
:102100000A6004339BB2B7E7012AB5D10A4A521AD2
:10211000E15C1160F5E7084959180A600433ACE73F
:10212000000004403C0004403800044034000440F7
:10213000300004400C00044000010440040004404E
:102140001000044014000440F7B5150080221C0064
:102150001023D2050091916807000B439360002380
:10216000654AD730136001F07FFD9D233E009B0040
:10217000F9583B00CA363200FC33002900D07FE01A
:10218000586801F0B9FE390032785C4BCB311A60E7
:102190004B780A781B0213438A78AC4612041A4320
:1021A000CB78281D1B061343554A1BBA13604B7985
:1021B0000A791B0213438A7912041A43CB791B064E
:1021C0001343504A1BBA13604B7A0A7A1B0213431B
:1021D0008A7A12041A43CB7A21001B0613434A4A17
:1021E0001BBA1360009A2B021343484A1360220063
:1021F000474B1B1B0093009BCE785B1801938B7899
:1022000036061B0433430E78043833434E780431CA
:1022100036023343019E33600328ECDC0321A80817
:10222000431C9B002940800003292BD13849E51825
:102230005E18A9786D78E35C09042D0229431943DF
:102240003160030008330021FF2B2DDD314B324973
:1022500019600F21314B1960012327490B60304B66
:1022600019680029FCD006211B680B40042B20D0E4
:1022700080220020D20593680A318B439360FEBD13
:1022800001217DE7022908D121495D18E11849782B
:10229000E35C090219432960D3E70129D3D11C4922
:1022A0005918E35C0B60CCE7194818180160043337
:1022B000CAE7002310490B606346002B0CDC3B008F
:1022C000FC335A68102101325A608022D20593688B
:1022D00001208B439360D2E7009B9B181B68190A6F
:1022E00013705170190C1B0ED37004235B42917054
:1022F0009C440432E0E7C046000004403C00044037
:102300003800044034000440300004400C00044015
:102310000001044004000440080F000010000440C5
:102320001400044070B5061E19D002225A4B9B7946
:102330009343012B13D1594B1A78FF2A0FD15A78A6
:10234000FF2A0CD19A78FF2A09D1DA78FF2A06D120
:102350001A79FF2A03D15B79FF2B00D199E0504B0A
:102360000C201A78012A08D000224E4D1A702978C4
:102370000B00093B042B01D8212070BD4B1F012B02
:10238000FAD9454CA37B042B00D982E0A279032A19
:1023900000D97EE09A1ED2B2012A02D860881F2896
:1023A00077D9002E56D0012E73D1A0880128E3D012
:1023B000002907D1581E032803D801F0B7FB1217D4
:1023C00015122E702978481E032811D80025364B87
:1023D0001D602823237501F01FFEA84227D0A58089
:1023E000CAE702212970EDE70421FBE70321F9E7A1
:1023F00007390129C0D82D490968C96A8906BBD5A2
:102400002B4908780028B7D1012A01D9002BB3D174
:1024100002230B708021274D2633890128782375EC
:1024200001F062FD80212878890101F0FDFD012382
:10243000A380214B1B78002B0AD0FA2280211F4B4E
:1024400092001B8809025A431A4B187801F0ACFB22
:10245000002092E701F078FD2B78A680073B012B46
:1024600003D917482E7001F097FD114B114C1A78C3
:10247000002A06D080210022207889011A7001F0FC
:1024800033FD01F021FC80212078090201F02CFDB0
:10249000DEE7122071E7C046A60BFF1F6B09FF1F86
:1024A0001A09FF1F1C09FF1F4809FF1F4064FF1F77
:1024B0002309FF1F1B09FF1F2109FF1F2C09FF1FF5
:1024C0000010004010B5002901D001F09DFD10BDA5
:1024D000F7B5604B01919978A1239B004B435E4A6D
:1024E000060014681022E418D6235B00E058362357
:1024F000FF33E35C00279343222B41D1574B0F3A24
:102500001A600760012501F0B7FC019B1880E823E1
:102510005B00E35C002B01D0B34258DD0023504F39
:10252000FB70AD33FF33E3581A68002A03D09B8851
:10253000DB439B071DD03823FF33E35C002B18D00F
:102540009B235B00E35C002B13D1D133FF33E35CAF
:10255000B3420EDAA4235B00E15AE018090A023103
:1025600001F042FC23000122FE33013E01351A87AF
:10257000FA70E8235B00E35C002B2AD0A8B2FEBD12
:1025800003683D00002BBED081880430090A023167
:1025900001F02AFCD6235B00E3581F60B2E723005A
:1025A000B133BA00FF339858013781880430090AE3
:1025B000023101F019FCE8235B00E35CBB42EEDC76
:1025C000E822F61AED1800235200A354A6E70027CC
:1025D000F1E7200001F0B0FB00281FD0002E1DDD28
:1025E0007319882647190193B600200001F03CFCBE
:1025F0005A30800020184068013581880430090A6B
:10260000023101F0F1FB200001F0B6FCA3590133C7
:10261000A351BD4202D0019B9D42E6D1114BE35C28
:10262000002BABD095239B00E35C002BA6D00E4B78
:10263000E15A0029A2D00D4AA35C994202D9013384
:10264000A3549BE700231A212000A35401F084FC2B
:1026500094E7C046300DFF1F3409FF1F00140340EC
:10266000E010FF1F5A020000720200005E0200002C
:102670000D4970B54A6E0D4CD2038B69D20BA24244
:1026800006D80B4D0224AA4204D901F0C5FA70BD48
:1026900002246442E21815007E2425402242F4D030
:1026A000A3432B438B61F0E700F000400A200000B9
:1026B000FC1C0000F8B51D4B1D4F1A78002A10D1E4
:1026C000BA7B002A02D101321A7003E0032AFAD041
:1026D000022AF8D001F0A0FC00220120154B1A704C
:1026E000F8BD154B154D1C68154B9E7801232B70BA
:1026F0002878C0B200F0A2FBBB7B002B0BD101F00D
:102700007BFBA1239B007343E41883239B00E41805
:1027100023782B70E4E7032B02D101F025FBF0E7CF
:102720000020022BDCD101F0D7FAEAE71C09FF1FD9
:10273000A60BFF1F2309FF1F3409FF1F490AFF1FB4
:10274000300DFF1FF0B587B00EAD2F780FAD2D788F
:102750000593AC46634614000E4D0CAA12782E78F1
:1027600003930D9B009201932200059B029701F0B9
:10277000BBFA2E70012C01D0042C08D1802206490E
:102780008B889343054A1278D20113438B8007B09C
:10279000F0BDC0461C09FF1F6C11FF1F7809FF1F09
:1027A0000B001B3B70B504003020E02B0DD813004C
:1027B000E025493BFF3B9BB2ED00AB4205D8034B04
:1027C000200019825A8201F05FFB70BD8410FF1F48
:1027D00010B501F051FA054B00205B68052B04D9B8
:1027E000034A5268D20200D4980810BD001000407D
:1027F000FCE100E070B501F0A7FB0D4B1B68FC335A
:10280000DC691D6AFFF7E4FF6419844204D2094BB6
:1028100001241B68002B07D004220024064B1A70E9
:10282000064A93690133936101F04EFA200070BDAE
:102830004064FF1F9809FF1F2309FF1FFC0FFF1FA4
:1028400070B50C4D2B68FC335C6A01F07DFBFFF723
:10285000BFFF2B680025FC339B6AE318834204D238
:10286000054B1B68AB4200D1051B01F02DFA280077
:1028700070BDC0464064FF1F9809FF1FD722044B5C
:1028800092009B5810B5002B00D0984710BDC04651
:102890000000FF1F10B501F0D3F8FFF7EFFF274945
:1028A000274BCA6D274C1A4084235B001343CB652A
:1028B000254B1B68186A01F0BFFA244B244A1A60A2
:1028C000244B254A1A60A022244B52001A60244B44
:1028D000187801F041FA2000224901F0ADFB0023F5
:1028E000A3600233A360204B2049236003232048C8
:1028F000A36001F0A1FB10221E4BFF201A60802272
:1029000052031A60802292031A60802212041A6015
:1029100001F05AFA012001F097F9FA20400001F085
:1029200013FA582001F020FB134801F0ADF9012003
:1029300001F022F9072001F0F7F910BD00F0004086
:1029400000FEFEFF141000404064FF1F0000034023
:102950000180063DBC00034034080000A400034091
:102960004A0AFF1F71020000C3090000FFFF3F0079
:102970002810004000E100E030750000674E336829
:1029800088331B6883F3088801F036FB644A654985
:10299000136800200B401360634B644A1B6893422A
:1029A00000D1A6E001F0F0F90221614A13688B43DF
:1029B0001360FFF76FFF5F4B5F4C1878C0B201F0F8
:1029C0000BF90023A3600233A3605C4B012023605A
:1029D00001F032FA0323A36001F0E6FA040001F0EB
:1029E0004BF9050001F0E0FA554B186001F064FA6C
:1029F000544B1968621A531EA14200D21300802260
:102A0000D203934201D39B029B0A3268D16AC90761
:102A100000D471E04C491C0C09689BB24C435943EB
:102A20002402090A641803264849FC3293680A689C
:102A300047489B1A474A0768126847499B18474A04
:102A40009A1833409208DB190A600360042B03D9FB
:102A5000013233400A6003600E684149A619300014
:102A600001F0AAF83F4F3E493B68C3183B60300075
:102A7000019301F0B9F83C4E3068081838493060CD
:102A8000884205D9019B01333B6001F0ADF831600C
:102A900001F022FA354B1B78002B0DD001F0ECF839
:102AA000334B621B196812188A4232D24919091B2A
:102AB000091A304801F0C0FA2F4E337A002B0ED09D
:102AC00001F0DAF8621BF1681218914224D9491911
:102AD000091B091A294801F0AFFA00233372284B69
:102AE00083F3088801F028FA002001F04DF901F085
:102AF000B3F801F049F95CE7DC0199000234641A8B
:102B00005900641A09214B438033CB40A408E418D0
:102B100089E7FA218900CCE71A49DBE74064FF1F07
:102B20001CF00040FFFFC1FF0C0AFF1FB64121034C
:102B300010000040490AFF1F14100040C3090000A4
:102B4000100AFF1F340AFF1F380AFF1F200AFF1F49
:102B5000280AFF1F1C0AFF1F240AFF1FC4090000C8
:102B6000710200006008FF1F2C0AFF1F1C09FF1FD5
:102B7000E408FF1F00100040740BFF1F3C100040D2
:102B800000000020DC050000A022054B92009B58AD
:102B900010B5002B01D0984710BD01F055F9FBE7A7
:102BA0000000FF1FA122054B92009B5810B5002B7F
:102BB00001D0984710BD01F047F9FBE70000FF1F67
:102BC000A222054B92009B5810B5002B01D09847CC
:102BD00010BD01F039F9FBE70000FF1FA322054BF0
:102BE00092009B5810B5002B01D0984710BD01F002
:102BF0002BF9FBE70000FF1FA422054B92009B5816
:102C000010B5002B01D0984710BD01F01DF9FBE76E
:102C10000000FF1F70B501F02FF84F4B186000F057
:102C2000BBFF0400C30702D400F0E6FF70BD002222
:102C30004A4B1A604A4B18780138042829D800F00A
:102C400075FF0320181C2400200001F0DDF8012886
:102C5000ECD0444C2378042B6ED101F09DF8002871
:102C6000E4D001F0D9F8582001F07EF90223237056
:102C7000DCE7200000F0A8FFE9E7200001F0ECF914
:102C8000E5E7200000F0C0FFE1E7200000F0CCFF06
:102C9000DDE701F0A9F90500012808D1324B1B78C6
:102CA000053B012B03D82000FFF76EFFD1E72D4B2A
:102CB0001B78022B01D0052B20D1022D28D12B4BC4
:102CC0009B7BAB431CD12000FFF76CFF264B187891
:102CD0000128BED16405BCD4244925224B7B034284
:102CE00005D1233A13405A42534126331A000B7D33
:102CF0009342AED9322001F06FF8AAE7022D07D136
:102D0000194B1B78052B11D12000FFF759FFDDE788
:102D1000012D0BD1012B03D12000FFF75FFF98E7B6
:102D2000062B03D12000FFF767FF92E7200001F098
:102D30008BF8022D8DD1C9E7032B04D10C4B987C65
:102D400000F0BAFF72E7072B00D06FE7094B987BC2
:102D500000F002FF6AE7C0469C09FF1F9809FF1FA9
:102D60009009FF1F2309FF1F1C09FF1FA60BFF1F50
:102D7000BC0BFF1FD40BFF1FFA210A4B0A4A490064
:102D80001A640A4A5A500A4A04395A50094A083100
:102D90009A64094A5A50094A5C315A50084ADA661C
:102DA0007047C0460000FF1F4527FF1F4128FF1F37
:102DB000F527FF1F2523FF1FB526FF1FC51DFF1F7A
:102DC000991DFF1F10B500F099FE10BDF7B50B0C53
:102DD000FF270122009300233C001E001D009446A3
:102DE000019089B262469A40100008401841361896
:102DF000B6B2FF2F02D1012E00D19FB2009802403F
:102E00001A41AD18ADB2FF2C02D1012D00D19CB2F8
:102E10000133102BE6D10320012E07D1012D04D15F
:102E2000019B2401E4191C700138FEBD102EFCD159
:102E30000238102DF9D00230F7E700008023F7B5F3
:102E40009C46264B264F01932649274A274D284C5E
:102E5000284B02281AD1604638600868264E304058
:102E6000802636033043086001990978002909D18A
:102E70001660224A2A60224A2260E02219689143A1
:102E8000A03A1BE08021C9021160F2E766463E606D
:102E90000F68194E3E408027FF023E430E600199A5
:102EA000097800290DD1176001280ED1154A2A6032
:102EB000154A2260E02219689143C03A0A431A6019
:102EC000F7BD802189021160EEE7E0210F4A02433D
:102ED0002A600F4A22601A688A43F0E74B0AFF1FF4
:102EE000E0000340D800034090000340000003408E
:102EF0005000034040000340FFFFE3FF0280063D17
:102F0000804508220180063D8066082200800698E0
:102F100080550822F8B51E4B80261A680020140040
:102F20003440324232D11A681A4F32431A600122B9
:102F30003B68063093433B6000F07EFF0122164D54
:102F40002B681E432E603B680A2613433B60802794
:102F5000BF00124B1B683B4211D1013EF6B2FF2E5F
:102F600009D17E220E4B1C682B68E40B144093435E
:102F700023432B6005E0082000F05EFFE9E7002E08
:102F8000EFD180222B68600893432B60F8BDC046C8
:102F9000C4F000405CF0004018F0004068F00040D1
:102FA00060F0004010B500F0E7FE01215820034A10
:102FB00000F07AFEFFF7AEFF10BDC046600AFF1FAB
:102FC00010B578220021034800F09EFE00F0DCFDE1
:102FD000002010BD4867FF1F70B5040000F0B4FF6B
:102FE00000230C200B4A010059438D18515C002925
:102FF0000DD0A14208D1012300246B7000F01CFE0B
:1030000000F062FE200070BD01330A2BEBD11224C8
:10301000F6E7C0464867FF1F70B5040000F094FF54
:10302000002319001D000D4A1078002806D0A04288
:103030000CD1557001310C320A29F5D1002B0AD17F
:1030400000F0A2FD00F040FE002070BD5078461E4A
:10305000B0411B18EEE700F0EFFDF3E74867FF1FF4
:10306000F7B504000C20002384460E4D01926746FC
:103070005F43E85D7E19A04212D000280BD10A4BB5
:103080009C4662461B7808331370019B70707C5518
:103090007160B360FEBD01330A2BE8D10320F9E76C
:1030A0000720F7E74867FF1F4467FF1F8020F8B538
:1030B000484BC0051B68C1248360474BFF251A6835
:1030C000012313434361454BA4001A68444B40213C
:1030D0001A60444B1A68444B1A60444B1A59AA436D
:1030E0001A51C52292009E58AE4331438026995012
:1030F0009F583F49F6010F403E439E509E588027FF
:103100003602360A3043985080201A5900020A408D
:1031100002431A5104341A59364E3F043240802675
:103120003A431A511A5936061202120A32431A51F8
:1031300008341A5980260A4002431A51C3229200C9
:103140009F58B446AF4337439F509F58294E0F4076
:1031500007439F509F5837408026360437438026C8
:103160009F509F5836063F023F0A37439F50C02268
:103170001F59AF433A431A511A591202120A164301
:10318000C6221E5192009C58AC4365462C439C506D
:103190009C5800250C4020439850C72080001A58A6
:1031A000154C1140C02212020A431A50134B1B78CF
:1031B000DB08AB4201DC0020F8BD2378002B06D0F1
:1031C000A368002B00D0984701350C34EEE712209D
:1031D000F2E7C0466443FF1F6043FF1FB0F00040AA
:1031E0004067FF1FB4F000403C67FF1F00E100E0B4
:1031F000FF00FFFFFFFF00FF4867FF1F4467FF1F3F
:10320000030010B51F2809D8072200201340072407
:1032100004490A78A24313430B7010BD0023062013
:10322000F5E7C0464467FF1F054B06491B780A684F
:1032300005485B0702401B0B134300200B607047DF
:103240004467FF1F1CF00040FFFFC1FF70B50C2555
:10325000FFF7EAFF0A4B1C780A4BE4086543ED18B8
:10326000002C01D1200070BD2B78002B06D06B689C
:10327000002B00D09847013C0C3DF1E71220F2E70B
:103280004467FF1F3C67FF1F1FB5002102220B0090
:1032900001910091052000F0DFFD02230B490A682F
:1032A0001A42FCD120230393039B5A1E0392002B46
:1032B000FAD1074A1368002BFCDA0B246C44200077
:1032C000012100F019FD207804B010BD90C8004025
:1032D00000C8004013B504000A4B0193019B002B6A
:1032E00001D1112016BDFFF7CFFF23000340044298
:1032F00005D0052000F0A0FD019B013BEDE7180083
:10330000F0E7C046FFFFFF0707B500F01DFE802273
:103310000821D205936A0191002B01D107399162EE
:1033200002210C4A11600199481E01900029FAD12E
:1033300003311160053101910199481E0190002966
:10334000FAD11160002B02D18022D205936200F0E5
:10335000BBFC07BD00C00040F0B52D4C89B0237800
:10336000002B4FD1FEF7CEFA02232A4F03903A6882
:103370001A42FCD120230693069B5A1E0692002B6C
:10338000FAD1254E3368002BFCDA0120FFF7A2FFAB
:10339000011E02D0112009B0F0BD030003220190EC
:1033A000009005AD9F2000F057FD0321280000F09C
:1033B000A3FC02233A681A42FCD120230793079BFF
:1033C0005A1E0792002BFAD13368002BFCDA012039
:1033D000FFF780FF0028DDD10398FEF7A7FAAA784F
:1033E0006B7811041B020B4329780B4363601300B5
:1033F000113B0A49052B07D801239340A3600B60BA
:10340000012323700020C6E780231B03F6E7C04694
:103410004C43FF1F90C8004000C800409808FF1FA1
:103420001E4B30B55A6818781D4B85B0D3185942D9
:103430004B4101210093002300F066FD194B1A4A0D
:1034400002259A6300221A6510325A658022C4212F
:103450009D65164B1648D202DA6789004258154B13
:1034600080241A4080231B041343435064234120CB
:103470000393E40500F006FA402000F003FA6562C9
:10348000039D6B1E0393002DFAD103236362FFF7A4
:103490003BFFA562FFF760FF05B030BD5843FF1F3B
:1034A00095FFFEF700C80040050001FF04E100E0C1
:1034B00000E100E0FFFF00FFF0B585B00700FEF778
:1034C00021FA022305002D4C22681A42FCD1202348
:1034D0000093009B5A1E0092002BFAD1284E3368AD
:1034E000002BFCDA0120FFF7F5FE002803D01124A1
:1034F000200005B0F0BD234B2360022322681A424E
:10350000FCD120230193019B5A1E0192002BFAD17A
:103510003368002BFCDA0120FFF7DCFE0028E6D13F
:10352000194B1F60022322681A42FCD12023029308
:10353000029B5A1E0292002BFAD13368002BFCDA50
:103540000120FFF7C7FE0028D1D1104B23600223D2
:1035500022681A42FCD120230393039B5A1E039234
:10356000002BFAD13368002BFCDA0120FFF7B2FE02
:10357000041EBCD12800FEF7D9F9B9E790C8004075
:1035800000C8004001000006A8C8004001800001FA
:1035900010B50020FFF790FF10BD000010B5064BDE
:1035A00018705960FFF73CFF00211320034AFFF712
:1035B00057FD002010BDC0465843FF1F2134FF1F98
:1035C000F0B5040085B003920291FEF79BF98822C2
:1035D00063035B0B52051A438023DB059D6A80233E
:1035E000274F0092BA68002601901B039A420CD91B
:1035F000F82326001B041E401C4206D08022214BCB
:1036000052025E6219680A431A60002D0BD100F065
:103610009BFC02221C4B1A608023DB055A62013A94
:103620009A6200F051FB0023039A934220D1002DAF
:103630000AD100F089FC144B03221D608023DB05B6
:103640005A629D6200F040FB8023BA681B039A42D5
:1036500008D9002E06D000220A4B0C495A621A687B
:103660000A401A600198FEF761F9002005B0F0BD2C
:10367000009A0299D2181278CA540133D4E7C0468E
:103680004C43FF1F00C8004000C00040FFFFFEFF8A
:10369000F0B587B0029103920400FEF733F9019070
:1036A00000F052FC802302250122234EDB05356009
:1036B0005D629A6200F008FB204F3B682B42FCD110
:1036C00020230493049B5A1E0492002BFAD11C4D14
:1036D0002B68002BFCDA0120FFF7FCFD002802D04C
:1036E000112007B0F0BD2000039A029900F06CFC95
:1036F000022304003A681A42FCD120230593059B5B
:103700005A1E0592002BFAD12B68002BFCDA0120FF
:10371000FFF7E0FD051EE3D100F016FC8023032235
:10372000DB0535605A629D6200F0CEFA0198FEF723
:10373000FDF8E0B2D5E7C04600C0004090C80040A8
:1037400000C80040F0B5802489B00600FEF7DAF822
:10375000E405A36A02250393029000F0F5FB012320
:10376000304F3D606562A36200F0AEFA2E4C2368D4
:103770002B42FCD120230593059B5A1E0592002B5A
:10378000FAD12A4D2B68002BFCDA0120FFF7A2FDAD
:10379000002803D01124200009B0F0BD244B236081
:1037A000022322681A42FCD120230693069B5A1E4C
:1037B0000692002BFAD12B68002BFCDA0120FFF7D0
:1037C00089FD021EE6D11B4B03211E600300019000
:1037D0000090202000F040FB022322681A42FCD116
:1037E00020230793079B5A1E0792002BFAD12B68C0
:1037F000002BFCDA0320FFF76DFD041ECAD100F098
:10380000A3FB80230322DB053C605A629C6200F02C
:103810005BFA039B002B01D1FFF776FD0298FEF7C0
:1038200085F8B8E700C0004090C8004000C80040DC
:103830000100000694C8004007B50002019104226F
:10384000000A01A9FFF724FF0EBD000073B50500B3
:1038500005240B4AA3005B429B1819686B46DE1DCA
:103860003000FFF7B3FA022804D133782B55013C1E
:10387000EFD276BD052CFCD00128FAD10230F8E752
:10388000140900111F2807D8012380228340D20584
:1038900091680B43936070473F2808D8012380222A
:1038A00020388340D20551690B435361F3E75F2809
:1038B000F1D80123802240388340D205116A0B439E
:1038C0001362E8E71F2807D8012280218240C9053A
:1038D0008B6893438B6070473F2808D80122802172
:1038E00020388240C9054B6993434B61F3E75F2859
:1038F000F1D80122802140388240C9050B6A9343E8
:103900000B62E8E71F2810D880230200DB05153A78
:103910001968012A06D820229143196019680A43C0
:103920001A60704701228240F6E73F2811D88023B1
:103930000200DB05353AD968032A06D810229143E4
:10394000D960D9680A43DA60EBE701222038824067
:10395000F5E75F28E5D842238022181A413B8340CF
:10396000D205516A99435162516A0B435362D8E7B9
:1039700010B50400012813D1A022184992050B6844
:103980005B015B0913430B60154B164A1968114024
:10399000154A0A431A60402219680A431A6010BD8A
:1039A0000028FCD101000A2000F0B6F921000B200C
:1039B00000F0B2F9C0220A4B920019680A43402174
:1039C0001A601A688A431A60B022044912060B680A
:1039D0005B015B0913430B60E1E7C04614F0004054
:1039E0001CF000407F00FEFF80FD010072B6074A18
:1039F0001368013313600422054B1A600023054A43
:103A000013608022D2055360FEE7C0467808FF1F8E
:103A1000C0F00040C4F0004005490B68002B05D100
:103A2000044A0A6004490A60044A13607047C046A9
:103A3000140AFF1F841E0000380AFF1FC4F0004054
:103A40000023034A1360034A1360034A136070475C
:103A500054F0004040F1004044F10040002310B514
:103A6000184C8AB0009301932378012B27D0694624
:103A7000012000F059FA002817D1009B1249029347
:103A8000019B06AA0393114B02A81B680493104BD9
:103A90001B68059300F088F910220E4906A800F073
:103AA000D3FA002804D1FF23237000200AB010BDF0
:103AB0000123094A074902A8237000F075F9012083
:103AC000F4E7C0464464FF1F1029001108290011C3
:103AD0000C290011202900114864FF1F13B501248F
:103AE0006946012000F020FA034B00940193FFF790
:103AF000B5FF200016BDC046BB0B000010B5FFF798
:103B00009FFFFFF7EBFF002802D0024B984710BD44
:103B1000FEE7C046E1A2000002B471464908490030
:103B2000095649008E4402BC7047C04602B4714633
:103B300049084900095C49008E4402BC7047C046F0
:103B400003B47146490840004900095A49008E44AF
:103B500003BC70470000000001B40248844601BC69
:103B6000604700BFC1F7000001B40248844601BCB1
:103B7000604700BF81B5001101B40248844601BC12
:103B8000604700BFE512010001B40248844601BC51
:103B9000604700BFADAE000001B40248844601BCDE
:103BA000604700BFBD0B010001B40248844601BC60
:103BB000604700BF8B52010001B40248844601BC3B
:103BC000604700BF090E000001B40248844601BCF2
:103BD000604700BF0934010001B40248844601BCBB
:103BE000604700BF8914010001B40248844601BC4B
:103BF000604700BF090E000001B40248844601BCC2
:103C0000604700BFDD0A010001B40248844601BCE0
:103C1000604700BFF535010001B40248844601BC8D
:103C2000604700BFD1AE000001B40248844601BC29
:103C3000604700BFF935010001B40248844601BC69
:103C4000604700BF21A9000001B40248844601BCBE
:103C5000604700BF6911010001B40248844601BCFD
:103C6000604700BF8552010001B40248844601BC90
:103C7000604700BF8944000001B40248844601BC8B
:103C8000604700BFC95C010001B40248844601BC22
:103C9000604700BF8D11010001B40248844601BC99
:103CA000604700BFE94C010001B40248844601BCF2
:103CB000604700BF0167010001B40248844601BCAF
:103CC000604700BF4DF9000001B40248844601BCC2
:103CD000604700BF9DA9000001B40248844601BCB2
:103CE000604700BF19FA000001B40248844601BCD5
:103CF000604700BF9D6A000001B40248844601BCD1
:103D0000604700BF3D71010001B40248844601BC18
:103D1000604700BFB70E000001B40248844601BCF2
:103D2000604700BFFDA1001101B40248844601BCF8
:103D3000604700BFF90D010001B40248844601BC90
:103D4000604700BF71B0000001B40248844601BC66
:103D5000604700BF8512010001B40248844601BCDF
:103D6000604700BFEDA5000001B40248844601BCD5
:103D7000604700BF75F8000001B40248844601BCEA
:103D8000604700BFED68010001B40248844601BCF1
:103D9000604700BF016C010001B40248844601BCC9
:103DA000604700BF01D7000001B40248844601BC4F
:103DB000604700BFDD3F000001B40248844601BCFB
:103DC000604700BF6D0B010001B40248844601BC8E
:103DD000604700BFED6B010001B40248844601BC9E
:103DE000604700BF6137010001B40248844601BC4E
:103DF000604700BFC115010001B40248844601BC00
:103E0000604700BFE9F6000001B40248844601BCE7
:103E1000604700BF0134010001B40248844601BC80
:103E2000604700BF6DF6000001B40248844601BC43
:103E3000604700BFBD5C010001B40248844601BC7C
:103E4000604700BF0189000001B40248844601BCFC
:103E5000604700BFE917010001B40248844601BC75
:103E6000604700BF496D010001B40248844601BCAF
:103E7000604700BFD9B0000001B40248844601BCCD
:103E8000604700BFCD0C010001B40248844601BC6C
:103E9000604700BF116E000001B40248844601BCB7
:103EA000604700BF85C1000001B40248844601BCE0
:103EB000604700BFE90B010001B40248844601BC21
:103EC000604700BFC166010001B40248844601BCDE
:103ED000604700BFE927000001B40248844601BCE6
:103EE000604700BFD544010001B40248844601BCCC
:103EF000604700BFB352010001B40248844601BCD0
:103F0000604700BF2144000001B40248844601BC60
:103F1000604700BFC56D010001B40248844601BC82
:103F2000604700BF8D82000001B40248844601BC96
:103F3000604700BFE1AC000001B40248844601BC08
:103F4000604700BF7997000001B40248844601BC75
:103F5000604700BF75A9000001B40248844601BC57
:103F6000604700BF53B9000001B40248844601BC59
:103F7000604700BF7912010001B40248844601BCC9
:103F8000604700BF5976010001B40248844601BC75
:103F9000604700BF51B8000001B40248844601BC2C
:103FA000604700BFC1A5000001B40248844601BCBF
:103FB000604700BF156B010001B40248844601BC94
:103FC000604700BFF9ED000001B40248844601BC1F
:103FD000604700BF9573010001B40248844601BCEC
:103FE000604700BF8937010001B40248844601BC24
:103FF000604700BFDD0C010001B40248844601BCEB
:10400000604700BFC9A9000001B40248844601BC52
:10401000604700BFE9D4000001B40248844601BCF7
:10402000604700BFA9D8000001B40248844601BC23
:10403000604700BF0D52010001B40248844601BC34
:10404000604700BF2D6C010001B40248844601BCEA
:10405000604700BFCD4C010001B40248844601BC5A
:08406000604700BF05340100B8
:104068000200000036BE00110100000048BC00112B
:104078000200000032BE001101000000A840FF1F2E
:104088000200000050BC001101000000BC61FF1FCD
:104098000200000030BE0011030000003061FF1F65
:1040A800120000000200000036BE001101000000EE
:1040B80090BC00110200000032BE00110100000097
:1040C8008DBC0011020000009ABC00110300000022
:1040D8006B61FF1F0200000030BE001103000000EA
:1040E8008061FF1F0200000032BE001101000000C5
:1040F8008CBC00110200000098BC001103000000F5
:104108004161FF1F0200000030BE001103000000E3
:104118006261FF1F0200000036BE001101000000AE
:10412800D0BC00110200000032BE001101000000E6
:10413800F141FF1F02000000E2BC00110100000075
:10414800CBBC00110200000032BE001101000000CB
:10415800F041FF1F02000000E0BC00110100000058
:104168008861FF1F0200000032BE0011010000003C
:10417800EF41FF1F02000000DEBC0011010000003B
:10418800BBBC00110200000032BE0011010000009B
:10419800EE41FF1F02000000DCBC0011010000001E
:1041A800B6BC00110200000032BE00110100000080
:1041B800ED41FF1F02000000DABC00110100000001
:1041C800B1BC00110200000032BE00110100000065
:1041D800EC41FF1F02000000D8BC001101000000E4
:1041E800ACBC001102020202020200000000000042
:1041F8000D0C0000A54B00116B4B001124BD0011E4
:1042080090011D0018001800FFFF070102030405B4
:104218000602010600000000000000000000000087
:104228000000000000000000000000000000000086
:10423800030000000200000036BE0011010000006B
:1042480044BD00110200000032BE00110100000050
:10425800AC42FF1F020000004EBD0011010000002B
:10426800B661FF1F0200000030BE0011030000000D
:104278002064FF1F0200000032BE00110100000090
:10428800AC42FF1F020000004CBD001101000000FD
:10429800B861FF1F0200000030BE001103000000DB
:1042A8001864FF1F126C6C6C00000000005800407E
:1042B800151600000001000000000111FFFF0000BA
:1042C8005048593600000000000000000B000500AF
:1042D800F0000000B4000028002800283075A00075
:1042E800A000A000A00000080008E001F0001000F5
:1042F8001000100010001000100050005000500076
:1043080010001000D0070000000000000F0001009E
:104318000500307507001000010081FF0000000053
:10432800FF000000E5730011ED7100117D6F0011B1
:10433800FFFF0100FF000000019E00117D9B00119E
:10434800959A00110000000000000000000008001D
:10435800040000003B0001085902E0018821280000
:10436800FF0000000200000036BE0011010000003E
:10437800FCBE00110200000032BE00110100000066
:10438800E943FF1F020000002EBE001101000000DB
:104398000068FF1F0200000032BE0011010000008B
:1043A800E843FF1F020000002CBE001101000000BE
:1043B800E643FF1F0200000032BE001101000000AA
:1043C800E443FF1F020000002ABE001101000000A4
:1043D800DC43FF1F180018001D00900102000003B5
:1043E800020200000200000036BE001101000000B9
:1043F80010BF00110200000032BE001101000000D1
:104408002C44FF1F0200000028BE0011000000001D
:10441800000000000200000030BE00110300000090
:064428002068FF1F20FFC9
:040000051FFF184180
:00000001FF
